 FARCmds

 Timestamp is 56b152f2 (Wed Feb 03 04:08:02 2016)

 Preferred load address is 10000000

 Start         Length     Name                   Class
 0001:00000000 00000198H .idata$5                CODE
 0001:00000198 00000004H .CRT$XCA                CODE
 0001:0000019c 00000004H .CRT$XCZ                CODE
 0001:000001a0 00000004H .CRT$XIA                CODE
 0001:000001a4 0000000cH .CRT$XIC                CODE
 0001:000001b0 00000004H .CRT$XIZ                CODE
 0001:000001b4 00000004H .CRT$XPA                CODE
 0001:000001b8 00000004H .CRT$XPZ                CODE
 0001:000001bc 00000004H .CRT$XTA                CODE
 0001:000001c0 00000004H .CRT$XTZ                CODE
 0001:000001c8 00002420H .rdata                  CODE
 0001:000025e8 000000dcH .rdata$r                CODE
 0001:000026d0 0000000cH .rdata$sxdata           CODE
 0001:000026dc 00000004H .rtc$IAA                CODE
 0001:000026e0 00000004H .rtc$IZZ                CODE
 0001:000026e4 00000004H .rtc$TAA                CODE
 0001:000026e8 00000004H .rtc$TZZ                CODE
 0001:000026f0 00009d39H .text                   CODE
 0001:0000c429 00000014H .text$yd                CODE
 0001:0000c440 00000224H .xdata$x                CODE
 0001:0000c664 00000064H .idata$2                CODE
 0001:0000c6c8 00000014H .idata$3                CODE
 0001:0000c6dc 00000198H .idata$4                CODE
 0001:0000c874 00000750H .idata$6                CODE
 0001:0000cfd0 000000a5H .edata                  CODE
 0002:00000000 00000c30H .data                   DATA
 0002:00000c40 000023c0H .bss                    DATA
 0003:00000000 00000058H .rsrc$01                DATA
 0003:00000060 00000378H .rsrc$02                DATA

  Address         Publics by Value              Rva+Base       Lib:Object

 0000:00000000       __except_list              00000000     <absolute>
 0000:00000003       ___safe_se_handler_count   00000003     <absolute>
 0000:00000000       ___ImageBase               10000000     <linker-defined>
 0001:00000000       __imp__RegQueryValueExW@24 10001000     advapi32:ADVAPI32.dll
 0001:00000004       __imp__RegCloseKey@4       10001004     advapi32:ADVAPI32.dll
 0001:00000008       __imp__IsTextUnicode@12    10001008     advapi32:ADVAPI32.dll
 0001:0000000c       __imp__RegOpenKeyExW@20    1000100c     advapi32:ADVAPI32.dll
 0001:00000010       \177ADVAPI32_NULL_THUNK_DATA 10001010     advapi32:ADVAPI32.dll
 0001:00000014       __imp__GetConsoleAliasesW@12 10001014     kernel32:KERNEL32.dll
 0001:00000018       __imp__GetConsoleAliasesLengthW@4 10001018     kernel32:KERNEL32.dll
 0001:0000001c       __imp__lstrcatW@8          1000101c     kernel32:KERNEL32.dll
 0001:00000020       __imp__GetLastError@0      10001020     kernel32:KERNEL32.dll
 0001:00000024       __imp__GetModuleFileNameW@12 10001024     kernel32:KERNEL32.dll
 0001:00000028       __imp__CloseHandle@4       10001028     kernel32:KERNEL32.dll
 0001:0000002c       __imp__ReadFile@20         1000102c     kernel32:KERNEL32.dll
 0001:00000030       __imp__CreateFileW@28      10001030     kernel32:KERNEL32.dll
 0001:00000034       __imp__MultiByteToWideChar@24 10001034     kernel32:KERNEL32.dll
 0001:00000038       __imp__GetACP@0            10001038     kernel32:KERNEL32.dll
 0001:0000003c       __imp__GetConsoleOutputCP@0 1000103c     kernel32:KERNEL32.dll
 0001:00000040       __imp__SetConsoleTitleW@4  10001040     kernel32:KERNEL32.dll
 0001:00000044       __imp__GetConsoleWindow@0  10001044     kernel32:KERNEL32.dll
 0001:00000048       __imp__GetCurrentDirectoryW@8 10001048     kernel32:KERNEL32.dll
 0001:0000004c       __imp__RemoveDirectoryW@4  1000104c     kernel32:KERNEL32.dll
 0001:00000050       __imp__DeleteFileW@4       10001050     kernel32:KERNEL32.dll
 0001:00000054       __imp__GetFileSize@8       10001054     kernel32:KERNEL32.dll
 0001:00000058       __imp__ExpandEnvironmentStringsW@12 10001058     kernel32:KERNEL32.dll
 0001:0000005c       __imp__Sleep@4             1000105c     kernel32:KERNEL32.dll
 0001:00000060       __imp__GetTempFileNameW@16 10001060     kernel32:KERNEL32.dll
 0001:00000064       __imp__CreateDirectoryW@8  10001064     kernel32:KERNEL32.dll
 0001:00000068       __imp__SearchPathW@24      10001068     kernel32:KERNEL32.dll
 0001:0000006c       __imp__GetEnvironmentVariableW@12 1000106c     kernel32:KERNEL32.dll
 0001:00000070       __imp__WaitForSingleObject@8 10001070     kernel32:KERNEL32.dll
 0001:00000074       __imp__CreateThread@24     10001074     kernel32:KERNEL32.dll
 0001:00000078       __imp__CreateProcessW@40   10001078     kernel32:KERNEL32.dll
 0001:0000007c       __imp__SetCurrentDirectoryW@4 1000107c     kernel32:KERNEL32.dll
 0001:00000080       __imp__SetConsoleCursorPosition@8 10001080     kernel32:KERNEL32.dll
 0001:00000084       __imp__GetConsoleScreenBufferInfo@8 10001084     kernel32:KERNEL32.dll
 0001:00000088       __imp__SetConsoleMode@8    10001088     kernel32:KERNEL32.dll
 0001:0000008c       __imp__GetConsoleMode@8    1000108c     kernel32:KERNEL32.dll
 0001:00000090       __imp__GetStdHandle@4      10001090     kernel32:KERNEL32.dll
 0001:00000094       __imp__GetFileAttributesW@4 10001094     kernel32:KERNEL32.dll
 0001:00000098       __imp__lstrlenW@4          10001098     kernel32:KERNEL32.dll
 0001:0000009c       __imp__lstrcpyW@8          1000109c     kernel32:KERNEL32.dll
 0001:000000a0       __imp__WriteConsoleW@20    100010a0     kernel32:KERNEL32.dll
 0001:000000a4       __imp__lstrcpynW@12        100010a4     kernel32:KERNEL32.dll
 0001:000000a8       __imp__GetStringTypeW@16   100010a8     kernel32:KERNEL32.dll
 0001:000000ac       __imp__LCMapStringW@24     100010ac     kernel32:KERNEL32.dll
 0001:000000b0       __imp__HeapSize@12         100010b0     kernel32:KERNEL32.dll
 0001:000000b4       __imp__LoadLibraryW@4      100010b4     kernel32:KERNEL32.dll
 0001:000000b8       __imp__HeapFree@12         100010b8     kernel32:KERNEL32.dll
 0001:000000bc       __imp__HeapAlloc@12        100010bc     kernel32:KERNEL32.dll
 0001:000000c0       __imp__HeapReAlloc@16      100010c0     kernel32:KERNEL32.dll
 0001:000000c4       __imp__GetCurrentThreadId@0 100010c4     kernel32:KERNEL32.dll
 0001:000000c8       __imp__DecodePointer@4     100010c8     kernel32:KERNEL32.dll
 0001:000000cc       __imp__GetCommandLineA@0   100010cc     kernel32:KERNEL32.dll
 0001:000000d0       __imp__IsProcessorFeaturePresent@4 100010d0     kernel32:KERNEL32.dll
 0001:000000d4       __imp__HeapCreate@12       100010d4     kernel32:KERNEL32.dll
 0001:000000d8       __imp__HeapDestroy@4       100010d8     kernel32:KERNEL32.dll
 0001:000000dc       __imp__GetProcAddress@8    100010dc     kernel32:KERNEL32.dll
 0001:000000e0       __imp__GetModuleHandleW@4  100010e0     kernel32:KERNEL32.dll
 0001:000000e4       __imp__ExitProcess@4       100010e4     kernel32:KERNEL32.dll
 0001:000000e8       __imp__WriteFile@20        100010e8     kernel32:KERNEL32.dll
 0001:000000ec       __imp__EncodePointer@4     100010ec     kernel32:KERNEL32.dll
 0001:000000f0       __imp__RaiseException@16   100010f0     kernel32:KERNEL32.dll
 0001:000000f4       __imp__GetCPInfo@8         100010f4     kernel32:KERNEL32.dll
 0001:000000f8       __imp__InterlockedIncrement@4 100010f8     kernel32:KERNEL32.dll
 0001:000000fc       __imp__InterlockedDecrement@4 100010fc     kernel32:KERNEL32.dll
 0001:00000100       __imp__GetOEMCP@0          10001100     kernel32:KERNEL32.dll
 0001:00000104       __imp__IsValidCodePage@4   10001104     kernel32:KERNEL32.dll
 0001:00000108       __imp__TlsAlloc@0          10001108     kernel32:KERNEL32.dll
 0001:0000010c       __imp__TlsGetValue@4       1000110c     kernel32:KERNEL32.dll
 0001:00000110       __imp__TlsSetValue@8       10001110     kernel32:KERNEL32.dll
 0001:00000114       __imp__TlsFree@4           10001114     kernel32:KERNEL32.dll
 0001:00000118       __imp__SetLastError@4      10001118     kernel32:KERNEL32.dll
 0001:0000011c       __imp__UnhandledExceptionFilter@4 1000111c     kernel32:KERNEL32.dll
 0001:00000120       __imp__SetUnhandledExceptionFilter@4 10001120     kernel32:KERNEL32.dll
 0001:00000124       __imp__IsDebuggerPresent@0 10001124     kernel32:KERNEL32.dll
 0001:00000128       __imp__TerminateProcess@8  10001128     kernel32:KERNEL32.dll
 0001:0000012c       __imp__GetCurrentProcess@0 1000112c     kernel32:KERNEL32.dll
 0001:00000130       __imp__SetHandleCount@4    10001130     kernel32:KERNEL32.dll
 0001:00000134       __imp__InitializeCriticalSectionAndSpinCount@8 10001134     kernel32:KERNEL32.dll
 0001:00000138       __imp__GetFileType@4       10001138     kernel32:KERNEL32.dll
 0001:0000013c       __imp__GetStartupInfoW@4   1000113c     kernel32:KERNEL32.dll
 0001:00000140       __imp__DeleteCriticalSection@4 10001140     kernel32:KERNEL32.dll
 0001:00000144       __imp__GetModuleFileNameA@12 10001144     kernel32:KERNEL32.dll
 0001:00000148       __imp__FreeEnvironmentStringsW@4 10001148     kernel32:KERNEL32.dll
 0001:0000014c       __imp__WideCharToMultiByte@32 1000114c     kernel32:KERNEL32.dll
 0001:00000150       __imp__GetEnvironmentStringsW@0 10001150     kernel32:KERNEL32.dll
 0001:00000154       __imp__QueryPerformanceCounter@4 10001154     kernel32:KERNEL32.dll
 0001:00000158       __imp__GetTickCount@0      10001158     kernel32:KERNEL32.dll
 0001:0000015c       __imp__GetCurrentProcessId@0 1000115c     kernel32:KERNEL32.dll
 0001:00000160       __imp__GetSystemTimeAsFileTime@4 10001160     kernel32:KERNEL32.dll
 0001:00000164       __imp__LeaveCriticalSection@4 10001164     kernel32:KERNEL32.dll
 0001:00000168       __imp__EnterCriticalSection@4 10001168     kernel32:KERNEL32.dll
 0001:0000016c       __imp__RtlUnwind@16        1000116c     kernel32:KERNEL32.dll
 0001:00000170       \177KERNEL32_NULL_THUNK_DATA 10001170     kernel32:KERNEL32.dll
 0001:00000174       __imp__UuidFromStringW@8   10001174     rpcrt4:RPCRT4.dll
 0001:00000178       \177RPCRT4_NULL_THUNK_DATA 10001178     rpcrt4:RPCRT4.dll
 0001:0000017c       __imp__GetWindowTextLengthW@4 1000117c     user32:USER32.dll
 0001:00000180       __imp__GetWindowTextW@12   10001180     user32:USER32.dll
 0001:00000184       \177USER32_NULL_THUNK_DATA 10001184     user32:USER32.dll
 0001:00000188       __imp__CoCreateInstance@20 10001188     ole32:ole32.dll
 0001:0000018c       __imp__CoUninitialize@0    1000118c     ole32:ole32.dll
 0001:00000190       __imp__CoInitialize@4      10001190     ole32:ole32.dll
 0001:00000194       \177ole32_NULL_THUNK_DATA  10001194     ole32:ole32.dll
 0001:00000198       ___xc_a                    10001198     LIBCMT:crt0init.obj
 0001:0000019c       ___xc_z                    1000119c     LIBCMT:crt0init.obj
 0001:000001a0       ___xi_a                    100011a0     LIBCMT:crt0init.obj
 0001:000001b0       ___xi_z                    100011b0     LIBCMT:crt0init.obj
 0001:000001b4       ___xp_a                    100011b4     LIBCMT:crt0init.obj
 0001:000001b8       ___xp_z                    100011b8     LIBCMT:crt0init.obj
 0001:000001bc       ___xt_a                    100011bc     LIBCMT:crt0init.obj
 0001:000001c0       ___xt_z                    100011c0     LIBCMT:crt0init.obj
 0001:000001c8       ??_C@_1BE@KBOCGMKN@?$AAS?$AAe?$AAp?$AAa?$AAr?$AAa?$AAt?$AAo?$AAr?$AA?$AA@ 100011c8     FARCmds.obj
 0001:000001dc       ??_C@_1BI@BKNCFIOG@?$AAM?$AAa?$AAx?$AAD?$AAa?$AAt?$AAa?$AAS?$AAi?$AAz?$AAe?$AA?$AA@ 100011dc     FARCmds.obj
 0001:000001f4       ??_C@_1BK@LOJIPNKK@?$AAE?$AAd?$AAi?$AAt?$AAN?$AAe?$AAw?$AAF?$AAi?$AAl?$AAe?$AAs?$AA?$AA@ 100011f4     FARCmds.obj
 0001:00000210       ??_C@_1BM@BMDAMABJ@?$AAV?$AAi?$AAe?$AAw?$AAZ?$AAe?$AAr?$AAo?$AAF?$AAi?$AAl?$AAe?$AAs?$AA?$AA@ 10001210     FARCmds.obj
 0001:0000022c       ??_C@_1BE@EKEFMMPP@?$AAC?$AAa?$AAt?$AAc?$AAh?$AAM?$AAo?$AAd?$AAe?$AA?$AA@ 1000122c     FARCmds.obj
 0001:00000240       ??_C@_1BM@IEHCKIMD@?$AAS?$AAh?$AAo?$AAw?$AAC?$AAm?$AAd?$AAO?$AAu?$AAt?$AAp?$AAu?$AAt?$AA?$AA@ 10001240     FARCmds.obj
 0001:0000025c       _MainGuid                  1000125c     FARCmds.obj
 0001:0000026c       _ConfigMenuGuid            1000126c     FARCmds.obj
 0001:0000027c       _DialogGuid                1000127c     FARCmds.obj
 0001:0000028c       ??_C@_1DE@BGKMIKPD@?$AAE?$AAu?$AAg?$AAe?$AAn?$AAe?$AA?5?$AAR?$AAo?$AAs?$AAh?$AAa?$AAl?$AA?5?$AA?$CG?$AA?5?$AAF?$AAa?$AAr?$AA?5?$AAG?$AAr?$AAo?$AAu?$AAp?$AA?$AA@ 1000128c     FARCmds.obj
 0001:000002c0       ??_C@_1EI@IHKPBHMH@?$AAF?$AAA?$AAR?$AA?5?$AAC?$AAo?$AAm?$AAm?$AAa?$AAn?$AAd?$AAs?$AA?5?$AAP?$AAl?$AAu?$AAg?$AAi?$AAn?$AA?5?$AAf?$AAo?$AAr?$AA?5?$AAF?$AAa?$AAr?$AA?5?$AAM?$AAa?$AAn?$AAa@ 100012c0     FARCmds.obj
 0001:00000308       ??_C@_1BA@LGNBLCFH@?$AAF?$AAA?$AAR?$AAC?$AAm?$AAd?$AAs?$AA?$AA@ 10001308     FARCmds.obj
 0001:00000318       ??_C@_13HOIJIPNN@?$AA?5?$AA?$AA@ 10001318     FARCmds.obj
 0001:00000320       ??_C@_1GC@PBJAIBOO@?$AAv?$AAi?$AAe?$AAw?$AA?3?$AAe?$AAd?$AAi?$AAt?$AA?3?$AAg?$AAo?$AAt?$AAo?$AA?3?$AAc?$AAl?$AAi?$AAp?$AA?3?$AAw?$AAh?$AAe?$AAr?$AAe?$AAi?$AAs?$AA?3?$AAl?$AAi?$AAn?$AAk@ 10001320     FARCmds.obj
 0001:00000384       ??_7?$DialogItemBinding@UFarDialogItem@@@@6B@ 10001384     FARCmds.obj
 0001:0000038c       ??_7?$DialogBuilderBase@UFarDialogItem@@@@6B@ 1000138c     FARCmds.obj
 0001:000003b0       ??_C@_15EFLNJKHH@?$AA?$CF?$AAu?$AA?$AA@ 100013b0     FARCmds.obj
 0001:000003b8       ??_7PluginUIntEditFieldBinding@@6B@ 100013b8     FARCmds.obj
 0001:000003c0       ??_7PluginDialogBuilder@@6B@ 100013c0     FARCmds.obj
 0001:000003e4       ??_7PluginCheckBoxBinding@@6B@ 100013e4     FARCmds.obj
 0001:000003ec       ??_7PluginRadioButtonBinding@@6B@ 100013ec     FARCmds.obj
 0001:000003f4       ??_7PluginIntEditFieldBinding@@6B@ 100013f4     FARCmds.obj
 0001:000003fc       ??_C@_11LOCGONAA@?$AA?$AA@ 100013fc     FARCmds.obj
 0001:00000400       ??_C@_1O@BJPKKLLM@?$AAC?$AAo?$AAn?$AAf?$AAi?$AAg?$AA?$AA@ 10001400     FARCmds.obj
 0001:00000410       ??_C@_15BNIPFGCG@?$AA$?$AA?$CK?$AA?$AA@ 10001410     Mix.obj
 0001:00000418       ??_C@_1BE@EKCMLKPN@?$AA?$CF?$AAC?$AAO?$AAM?$AAS?$AAP?$AAE?$AAC?$AA?$CF?$AA?$AA@ 10001418     Mix.obj
 0001:0000042c       ??_C@_0BC@KFCLBIA@?$AB?$BE?$AC?$AA?$AA?$AA?$AA?$AA?$MA?$AA?$AA?$AA?$AA?$AA?$AAF?$JL?$AA@ 1000142c     Mix.obj
 0001:00000440       ??_C@_13FPGAJAPJ@?$AA?2?$AA?$AA@ 10001440     OpenCmd.obj
 0001:00000444       ??_C@_1BE@BNONMOPA@?$AA?2?$AA?2?$AA?4?$AA?2?$AAc?$AAd?$AAr?$AAo?$AAm?$AA?$AA@ 10001444     OpenCmd.obj
 0001:00000458       ??_C@_1CE@JKDBMIKG@?$AA?2?$AA?2?$AA?4?$AA?2?$AAP?$AAh?$AAy?$AAs?$AAi?$AAc?$AAa?$AAl?$AAD?$AAr?$AAi?$AAv?$AAe?$AA?$AA@ 10001458     OpenCmd.obj
 0001:0000047c       ??_C@_19BKJMDJK@?$AA?2?$AA?2?$AA?4?$AA?2?$AA?$AA@ 1000147c     OpenCmd.obj
 0001:00000488       ??_C@_17IJMNDCL@?$AA?$CF?$AAl?$AAu?$AA?$AA@ 10001488     OpenCmd.obj
 0001:00000490       ??_C@_1BA@EIPEFBMB@?$AA?$CF?$AAl?$AAu?$AA?1?$AA?$CF?$AAl?$AAu?$AA?$AA@ 10001490     OpenCmd.obj
 0001:000004a8       ??_C@_1GK@PPEHOOAL@?$AAS?$AAO?$AAF?$AAT?$AAW?$AAA?$AAR?$AAE?$AA?2?$AAM?$AAi?$AAc?$AAr?$AAo?$AAs?$AAo?$AAf?$AAt?$AA?2?$AAW?$AAi?$AAn?$AAd?$AAo?$AAw?$AAs?$AA?2?$AAC?$AAu?$AAr?$AAr?$AAe@ 100014a8     OpenCmd.obj
 0001:00000514       ??_C@_13PJJBFPED@?$AA?$DL?$AA?$AA@ 10001514     OpenCmd.obj
 0001:00000518       ??_C@_1BA@HAHEJCII@?$AAP?$AAA?$AAT?$AAH?$AAE?$AAX?$AAT?$AA?$AA@ 10001518     OpenCmd.obj
 0001:00000528       ??_C@_19IJOJOJIB@?$AAP?$AAA?$AAT?$AAH?$AA?$AA@ 10001528     OpenCmd.obj
 0001:00000534       ??_C@_1BA@IBNPAI@?$AAF?$AAA?$AAR?$AAH?$AAO?$AAM?$AAE?$AA?$AA@ 10001534     OpenCmd.obj
 0001:00000544       ??_C@_15GBHPEJPD@?$AA?1?$AAS?$AA?$AA@ 10001544     OpenCmd.obj
 0001:0000054c       ??_C@_15MDAMMGLB@?$AA?1?$AAN?$AA?$AA@ 1000154c     OpenCmd.obj
 0001:00000554       ??_C@_19JMGCACDF@?$AA?1?$AAM?$AAS?$AAG?$AA?$AA@ 10001554     OpenCmd.obj
 0001:00000560       ??_C@_13NEIAEHFG@?$AA?$CC?$AA?$AA@ 10001560     OpenCmd.obj
 0001:00000564       ??_C@_1BM@MDBPDFDA@?$AA?$CF?$AAC?$AAO?$AAM?$AAS?$AAP?$AAE?$AAC?$AA?$CF?$AA?5?$AA?1?$AAc?$AA?5?$AA?$AA@ 10001564     OpenCmd.obj
 0001:00000580       ??_C@_1BC@ENICKDH@?$AAC?$AAo?$AAn?$AAt?$AAe?$AAn?$AAt?$AAs?$AA?$AA@ 10001580     OpenCmd.obj
 0001:00000594       ??_C@_17KKFGGCGH@?$AAR?$AAU?$AAN?$AA?$AA@ 10001594     OpenCmd.obj
 0001:0000059c       ??_C@_17NMIMIGP@?$AAR?$AAu?$AAn?$AA?$AA@ 1000159c     OpenCmd.obj
 0001:000005a4       ??_C@_19JHOCBEIE@?$AAV?$AAI?$AAE?$AAW?$AA?$AA@ 100015a4     OpenCmd.obj
 0001:000005b0       ??_C@_19MJAKNMNK@?$AAV?$AAi?$AAe?$AAw?$AA?$AA@ 100015b0     OpenCmd.obj
 0001:000005bc       ??_C@_19PEJAKIIO@?$AAC?$AAL?$AAI?$AAP?$AA?$AA@ 100015bc     OpenCmd.obj
 0001:000005c8       ??_C@_19KKHIGANA@?$AAC?$AAl?$AAi?$AAp?$AA?$AA@ 100015c8     OpenCmd.obj
 0001:000005d4       ??_C@_1BA@NBLHMMII@?$AAW?$AAH?$AAE?$AAR?$AAE?$AAI?$AAS?$AA?$AA@ 100015d4     OpenCmd.obj
 0001:000005e4       ??_C@_1BA@BCPLKBBA@?$AAW?$AAh?$AAe?$AAr?$AAe?$AAI?$AAs?$AA?$AA@ 100015e4     OpenCmd.obj
 0001:000005f4       ??_C@_19KFAJFECL@?$AAE?$AAD?$AAI?$AAT?$AA?$AA@ 100015f4     OpenCmd.obj
 0001:00000600       ??_C@_19PLOBJMHF@?$AAE?$AAd?$AAi?$AAt?$AA?$AA@ 10001600     OpenCmd.obj
 0001:0000060c       ??_C@_19MEMGFJJL@?$AAG?$AAO?$AAT?$AAO?$AA?$AA@ 1000160c     OpenCmd.obj
 0001:00000618       ??_C@_19JKCOJBMF@?$AAG?$AAo?$AAt?$AAo?$AA?$AA@ 10001618     OpenCmd.obj
 0001:00000624       ??_C@_19NHGGBNEB@?$AAL?$AAI?$AAN?$AAK?$AA?$AA@ 10001624     OpenCmd.obj
 0001:00000630       ??_C@_19IJIONFBP@?$AAL?$AAi?$AAn?$AAk?$AA?$AA@ 10001630     OpenCmd.obj
 0001:0000063c       ??_C@_19LIDMLGEF@?$AAL?$AAO?$AAA?$AAD?$AA?$AA@ 1000163c     OpenCmd.obj
 0001:00000648       ??_C@_19OGNEHOBL@?$AAL?$AAo?$AAa?$AAd?$AA?$AA@ 10001648     OpenCmd.obj
 0001:00000654       ??_C@_1O@PAPHGGOK@?$AAU?$AAN?$AAL?$AAO?$AAA?$AAD?$AA?$AA@ 10001654     OpenCmd.obj
 0001:00000664       ??_C@_1O@PJHDHGJM@?$AAU?$AAn?$AAl?$AAo?$AAa?$AAd?$AA?$AA@ 10001664     OpenCmd.obj
 0001:00000674       _IID_IShellLinkW           10001674     shell32:shguid.obj
 0001:00000684       _IID_IPersistFile          10001684     uuid:objidl_i.obj
 0001:00000694       _CLSID_ShellLink           10001694     uuid:shguids2.obj
 0001:000006a8       ??_7bad_alloc@std@@6B@     100016a8     LIBCMT:new.obj
 0001:000006b0       ??_C@_0P@GHFPNOJB@bad?5allocation?$AA@ 100016b0     LIBCMT:new.obj
 0001:000006c0       __pRawDllMain              100016c0     LIBCMT:dllcrt0.obj
 0001:000006c0       __pDefaultRawDllMain       100016c0     LIBCMT:dllcrt0.obj
 0001:000006c4       ??_C@_0P@MIGLKIOC@CorExitProcess?$AA@ 100016c4     LIBCMT:crt0dat.obj
 0001:000006d4       ??_C@_1BI@BGOHAHKC@?$AAm?$AAs?$AAc?$AAo?$AAr?$AAe?$AAe?$AA?4?$AAd?$AAl?$AAl?$AA?$AA@ 100016d4     LIBCMT:crt0dat.obj
 0001:000006ec       ??_C@_1BO@BKOMIGKJ@?$AAr?$AAu?$AAn?$AAt?$AAi?$AAm?$AAe?$AA?5?$AAe?$AAr?$AAr?$AAo?$AAr?$AA?5?$AA?$AA@ 100016ec     LIBCMT:crt0msg.obj
 0001:0000070c       ??_C@_15JNBOKNOG@?$AA?$AN?$AA?6?$AA?$AA@ 1000170c     LIBCMT:crt0msg.obj
 0001:00000714       ??_C@_1BM@JBBEPPHI@?$AAT?$AAL?$AAO?$AAS?$AAS?$AA?5?$AAe?$AAr?$AAr?$AAo?$AAr?$AA?$AN?$AA?6?$AA?$AA@ 10001714     LIBCMT:crt0msg.obj
 0001:00000730       ??_C@_1BK@KMOMNAAI@?$AAS?$AAI?$AAN?$AAG?$AA?5?$AAe?$AAr?$AAr?$AAo?$AAr?$AA?$AN?$AA?6?$AA?$AA@ 10001730     LIBCMT:crt0msg.obj
 0001:0000074c       ??_C@_1BO@BFCDCGC@?$AAD?$AAO?$AAM?$AAA?$AAI?$AAN?$AA?5?$AAe?$AAr?$AAr?$AAo?$AAr?$AA?$AN?$AA?6?$AA?$AA@ 1000174c     LIBCMT:crt0msg.obj
 0001:00000770       ??_C@_1BOO@KGEDBGAJ@?$AAR?$AA6?$AA0?$AA3?$AA3?$AA?$AN?$AA?6?$AA?9?$AA?5?$AAA?$AAt?$AAt?$AAe?$AAm?$AAp?$AAt?$AA?5?$AAt?$AAo?$AA?5?$AAu?$AAs?$AAe?$AA?5?$AAM?$AAS?$AAI?$AAL?$AA?5?$AAc?$AAo?$AAd@ 10001770     LIBCMT:crt0msg.obj
 0001:00000960       ??_C@_1GG@GOPILAJP@?$AAR?$AA6?$AA0?$AA3?$AA2?$AA?$AN?$AA?6?$AA?9?$AA?5?$AAn?$AAo?$AAt?$AA?5?$AAe?$AAn?$AAo?$AAu?$AAg?$AAh?$AA?5?$AAs?$AAp?$AAa?$AAc?$AAe?$AA?5?$AAf?$AAo?$AAr?$AA?5?$AAl?$AAo@ 10001960     LIBCMT:crt0msg.obj
 0001:000009c8       ??_C@_1MG@ENCOOIDF@?$AAR?$AA6?$AA0?$AA3?$AA1?$AA?$AN?$AA?6?$AA?9?$AA?5?$AAA?$AAt?$AAt?$AAe?$AAm?$AAp?$AAt?$AA?5?$AAt?$AAo?$AA?5?$AAi?$AAn?$AAi?$AAt?$AAi?$AAa?$AAl?$AAi?$AAz?$AAe?$AA?5?$AAt@ 100019c8     LIBCMT:crt0msg.obj
 0001:00000a90       ??_C@_1DO@BMFCDCD@?$AAR?$AA6?$AA0?$AA3?$AA0?$AA?$AN?$AA?6?$AA?9?$AA?5?$AAC?$AAR?$AAT?$AA?5?$AAn?$AAo?$AAt?$AA?5?$AAi?$AAn?$AAi?$AAt?$AAi?$AAa?$AAl?$AAi?$AAz?$AAe?$AAd?$AA?$AN?$AA?6?$AA?$AA@ 10001a90     LIBCMT:crt0msg.obj
 0001:00000ad0       ??_C@_1EK@HHFLMAOL@?$AAR?$AA6?$AA0?$AA2?$AA8?$AA?$AN?$AA?6?$AA?9?$AA?5?$AAu?$AAn?$AAa?$AAb?$AAl?$AAe?$AA?5?$AAt?$AAo?$AA?5?$AAi?$AAn?$AAi?$AAt?$AAi?$AAa?$AAl?$AAi?$AAz?$AAe?$AA?5?$AAh?$AAe@ 10001ad0     LIBCMT:crt0msg.obj
 0001:00000b20       ??_C@_1GK@MFGOKLAG@?$AAR?$AA6?$AA0?$AA2?$AA7?$AA?$AN?$AA?6?$AA?9?$AA?5?$AAn?$AAo?$AAt?$AA?5?$AAe?$AAn?$AAo?$AAu?$AAg?$AAh?$AA?5?$AAs?$AAp?$AAa?$AAc?$AAe?$AA?5?$AAf?$AAo?$AAr?$AA?5?$AAl?$AAo@ 10001b20     LIBCMT:crt0msg.obj
 0001:00000b90       ??_C@_1GK@MCAAGJMO@?$AAR?$AA6?$AA0?$AA2?$AA6?$AA?$AN?$AA?6?$AA?9?$AA?5?$AAn?$AAo?$AAt?$AA?5?$AAe?$AAn?$AAo?$AAu?$AAg?$AAh?$AA?5?$AAs?$AAp?$AAa?$AAc?$AAe?$AA?5?$AAf?$AAo?$AAr?$AA?5?$AAs?$AAt@ 10001b90     LIBCMT:crt0msg.obj
 0001:00000c00       ??_C@_1EM@MAADIHMB@?$AAR?$AA6?$AA0?$AA2?$AA5?$AA?$AN?$AA?6?$AA?9?$AA?5?$AAp?$AAu?$AAr?$AAe?$AA?5?$AAv?$AAi?$AAr?$AAt?$AAu?$AAa?$AAl?$AA?5?$AAf?$AAu?$AAn?$AAc?$AAt?$AAi?$AAo?$AAn?$AA?5?$AAc@ 10001c00     LIBCMT:crt0msg.obj
 0001:00000c50       ??_C@_1GK@FHCKBEFA@?$AAR?$AA6?$AA0?$AA2?$AA4?$AA?$AN?$AA?6?$AA?9?$AA?5?$AAn?$AAo?$AAt?$AA?5?$AAe?$AAn?$AAo?$AAu?$AAg?$AAh?$AA?5?$AAs?$AAp?$AAa?$AAc?$AAe?$AA?5?$AAf?$AAo?$AAr?$AA?5?$AA_?$AAo@ 10001c50     LIBCMT:crt0msg.obj
 0001:00000cc0       ??_C@_1FC@ECHBIFBC@?$AAR?$AA6?$AA0?$AA1?$AA9?$AA?$AN?$AA?6?$AA?9?$AA?5?$AAu?$AAn?$AAa?$AAb?$AAl?$AAe?$AA?5?$AAt?$AAo?$AA?5?$AAo?$AAp?$AAe?$AAn?$AA?5?$AAc?$AAo?$AAn?$AAs?$AAo?$AAl?$AAe?$AA?5@ 10001cc0     LIBCMT:crt0msg.obj
 0001:00000d18       ??_C@_1EC@JIBHAOPH@?$AAR?$AA6?$AA0?$AA1?$AA8?$AA?$AN?$AA?6?$AA?9?$AA?5?$AAu?$AAn?$AAe?$AAx?$AAp?$AAe?$AAc?$AAt?$AAe?$AAd?$AA?5?$AAh?$AAe?$AAa?$AAp?$AA?5?$AAe?$AAr?$AAr?$AAo?$AAr?$AA?$AN?$AA?6@ 10001d18     LIBCMT:crt0msg.obj
 0001:00000d60       ??_C@_1FK@BEOGODMC@?$AAR?$AA6?$AA0?$AA1?$AA7?$AA?$AN?$AA?6?$AA?9?$AA?5?$AAu?$AAn?$AAe?$AAx?$AAp?$AAe?$AAc?$AAt?$AAe?$AAd?$AA?5?$AAm?$AAu?$AAl?$AAt?$AAi?$AAt?$AAh?$AAr?$AAe?$AAa?$AAd?$AA?5@ 10001d60     LIBCMT:crt0msg.obj
 0001:00000dc0       ??_C@_1FI@LOGNIKDM@?$AAR?$AA6?$AA0?$AA1?$AA6?$AA?$AN?$AA?6?$AA?9?$AA?5?$AAn?$AAo?$AAt?$AA?5?$AAe?$AAn?$AAo?$AAu?$AAg?$AAh?$AA?5?$AAs?$AAp?$AAa?$AAc?$AAe?$AA?5?$AAf?$AAo?$AAr?$AA?5?$AAt?$AAh@ 10001dc0     LIBCMT:crt0msg.obj
 0001:00000e18       ??_C@_1EG@BEHAGFJD@?$AAR?$AA6?$AA0?$AA1?$AA0?$AA?$AN?$AA?6?$AA?9?$AA?5?$AAa?$AAb?$AAo?$AAr?$AAt?$AA?$CI?$AA?$CJ?$AA?5?$AAh?$AAa?$AAs?$AA?5?$AAb?$AAe?$AAe?$AAn?$AA?5?$AAc?$AAa?$AAl?$AAl?$AAe?$AAd@ 10001e18     LIBCMT:crt0msg.obj
 0001:00000e60       ??_C@_1FI@HONFMGBI@?$AAR?$AA6?$AA0?$AA0?$AA9?$AA?$AN?$AA?6?$AA?9?$AA?5?$AAn?$AAo?$AAt?$AA?5?$AAe?$AAn?$AAo?$AAu?$AAg?$AAh?$AA?5?$AAs?$AAp?$AAa?$AAc?$AAe?$AA?5?$AAf?$AAo?$AAr?$AA?5?$AAe?$AAn@ 10001e60     LIBCMT:crt0msg.obj
 0001:00000eb8       ??_C@_1FE@LLNEDJMD@?$AAR?$AA6?$AA0?$AA0?$AA8?$AA?$AN?$AA?6?$AA?9?$AA?5?$AAn?$AAo?$AAt?$AA?5?$AAe?$AAn?$AAo?$AAu?$AAg?$AAh?$AA?5?$AAs?$AAp?$AAa?$AAc?$AAe?$AA?5?$AAf?$AAo?$AAr?$AA?5?$AAa?$AAr@ 10001eb8     LIBCMT:crt0msg.obj
 0001:00000f10       ??_C@_1FK@PGACCAFB@?$AAR?$AA6?$AA0?$AA0?$AA2?$AA?$AN?$AA?6?$AA?9?$AA?5?$AAf?$AAl?$AAo?$AAa?$AAt?$AAi?$AAn?$AAg?$AA?5?$AAp?$AAo?$AAi?$AAn?$AAt?$AA?5?$AAs?$AAu?$AAp?$AAp?$AAo?$AAr?$AAt?$AA?5@ 10001f10     LIBCMT:crt0msg.obj
 0001:00001020       ??_C@_1EK@MBDPDCGA@?$AAM?$AAi?$AAc?$AAr?$AAo?$AAs?$AAo?$AAf?$AAt?$AA?5?$AAV?$AAi?$AAs?$AAu?$AAa?$AAl?$AA?5?$AAC?$AA?$CL?$AA?$CL?$AA?5?$AAR?$AAu?$AAn?$AAt?$AAi?$AAm?$AAe?$AA?5?$AAL?$AAi?$AAb@ 10002020     LIBCMT:crt0msg.obj
 0001:0000106c       ??_C@_15IABLJNFO@?$AA?6?$AA?6?$AA?$AA@ 1000206c     LIBCMT:crt0msg.obj
 0001:00001074       ??_C@_17LGKOMLJ@?$AA?4?$AA?4?$AA?4?$AA?$AA@ 10002074     LIBCMT:crt0msg.obj
 0001:0000107c       ??_C@_1CO@EAEJAADC@?$AA?$DM?$AAp?$AAr?$AAo?$AAg?$AAr?$AAa?$AAm?$AA?5?$AAn?$AAa?$AAm?$AAe?$AA?5?$AAu?$AAn?$AAk?$AAn?$AAo?$AAw?$AAn?$AA?$DO?$AA?$AA@ 1000207c     LIBCMT:crt0msg.obj
 0001:000010ac       ??_C@_1DE@JNGNBFGO@?$AAR?$AAu?$AAn?$AAt?$AAi?$AAm?$AAe?$AA?5?$AAE?$AAr?$AAr?$AAo?$AAr?$AA?$CB?$AA?6?$AA?6?$AAP?$AAr?$AAo?$AAg?$AAr?$AAa?$AAm?$AA?3?$AA?5?$AA?$AA@ 100020ac     LIBCMT:crt0msg.obj
 0001:000010e4       ??_7exception@std@@6B@     100020e4     LIBCMT:stdexcpt.obj
 0001:000010ec       ??_C@_0BC@EOODALEL@Unknown?5exception?$AA@ 100020ec     LIBCMT:stdexcpt.obj
 0001:00001104       ??_7type_info@@6B@         10002104     LIBCMT:typinfo.obj
 0001:00001128       ??_C@_1BC@GDGBMEMK@?$AAH?$AAH?$AA?3?$AAm?$AAm?$AA?3?$AAs?$AAs?$AA?$AA@ 10002128     LIBCMT:nlsdata2.obj
 0001:0000113c       ??_C@_1CI@KNAKOEBC@?$AAd?$AAd?$AAd?$AAd?$AA?0?$AA?5?$AAM?$AAM?$AAM?$AAM?$AA?5?$AAd?$AAd?$AA?0?$AA?5?$AAy?$AAy?$AAy?$AAy?$AA?$AA@ 1000213c     LIBCMT:nlsdata2.obj
 0001:00001164       ??_C@_1BC@IEBCMHCM@?$AAM?$AAM?$AA?1?$AAd?$AAd?$AA?1?$AAy?$AAy?$AA?$AA@ 10002164     LIBCMT:nlsdata2.obj
 0001:00001178       ??_C@_15CLMNNGEL@?$AAP?$AAM?$AA?$AA@ 10002178     LIBCMT:nlsdata2.obj
 0001:00001180       ??_C@_15ODEHAHHF@?$AAA?$AAM?$AA?$AA@ 10002180     LIBCMT:nlsdata2.obj
 0001:00001188       ??_C@_1BC@FEMKIFH@?$AAD?$AAe?$AAc?$AAe?$AAm?$AAb?$AAe?$AAr?$AA?$AA@ 10002188     LIBCMT:nlsdata2.obj
 0001:0000119c       ??_C@_1BC@BGLIFPF@?$AAN?$AAo?$AAv?$AAe?$AAm?$AAb?$AAe?$AAr?$AA?$AA@ 1000219c     LIBCMT:nlsdata2.obj
 0001:000011b0       ??_C@_1BA@EPANDLNG@?$AAO?$AAc?$AAt?$AAo?$AAb?$AAe?$AAr?$AA?$AA@ 100021b0     LIBCMT:nlsdata2.obj
 0001:000011c0       ??_C@_1BE@DKAAMBJL@?$AAS?$AAe?$AAp?$AAt?$AAe?$AAm?$AAb?$AAe?$AAr?$AA?$AA@ 100021c0     LIBCMT:nlsdata2.obj
 0001:000011d4       ??_C@_1O@PAHLKOAC@?$AAA?$AAu?$AAg?$AAu?$AAs?$AAt?$AA?$AA@ 100021d4     LIBCMT:nlsdata2.obj
 0001:000011e4       ??_C@_19BIFMLPCD@?$AAJ?$AAu?$AAl?$AAy?$AA?$AA@ 100021e4     LIBCMT:nlsdata2.obj
 0001:000011f0       ??_C@_19EPFLPGAP@?$AAJ?$AAu?$AAn?$AAe?$AA?$AA@ 100021f0     LIBCMT:nlsdata2.obj
 0001:000011fc       ??_C@_1M@GJNLMHFD@?$AAA?$AAp?$AAr?$AAi?$AAl?$AA?$AA@ 100021fc     LIBCMT:nlsdata2.obj
 0001:00001208       ??_C@_1M@IKEENEDF@?$AAM?$AAa?$AAr?$AAc?$AAh?$AA?$AA@ 10002208     LIBCMT:nlsdata2.obj
 0001:00001214       ??_C@_1BC@JGDDFFAM@?$AAF?$AAe?$AAb?$AAr?$AAu?$AAa?$AAr?$AAy?$AA?$AA@ 10002214     LIBCMT:nlsdata2.obj
 0001:00001228       ??_C@_1BA@EFMEIEBA@?$AAJ?$AAa?$AAn?$AAu?$AAa?$AAr?$AAy?$AA?$AA@ 10002228     LIBCMT:nlsdata2.obj
 0001:00001238       ??_C@_17EGKACKIF@?$AAD?$AAe?$AAc?$AA?$AA@ 10002238     LIBCMT:nlsdata2.obj
 0001:00001240       ??_C@_17BBDMLCIG@?$AAN?$AAo?$AAv?$AA?$AA@ 10002240     LIBCMT:nlsdata2.obj
 0001:00001248       ??_C@_17FNLKOI@?$AAO?$AAc?$AAt?$AA?$AA@ 10002248     LIBCMT:nlsdata2.obj
 0001:00001250       ??_C@_17HCHCOKMG@?$AAS?$AAe?$AAp?$AA?$AA@ 10002250     LIBCMT:nlsdata2.obj
 0001:00001258       ??_C@_17ICPELBCN@?$AAA?$AAu?$AAg?$AA?$AA@ 10002258     LIBCMT:nlsdata2.obj
 0001:00001260       ??_C@_17IJPCKHK@?$AAJ?$AAu?$AAl?$AA?$AA@ 10002260     LIBCMT:nlsdata2.obj
 0001:00001268       ??_C@_17KCJGOCPB@?$AAJ?$AAu?$AAn?$AA?$AA@ 10002268     LIBCMT:nlsdata2.obj
 0001:00001270       ??_C@_17PNNKMEED@?$AAM?$AAa?$AAy?$AA?$AA@ 10002270     LIBCMT:nlsdata2.obj
 0001:00001278       ??_C@_17LFPOIHDD@?$AAA?$AAp?$AAr?$AA?$AA@ 10002278     LIBCMT:nlsdata2.obj
 0001:00001280       ??_C@_17CKNLEDEC@?$AAM?$AAa?$AAr?$AA?$AA@ 10002280     LIBCMT:nlsdata2.obj
 0001:00001288       ??_C@_17LMDJEKJN@?$AAF?$AAe?$AAb?$AA?$AA@ 10002288     LIBCMT:nlsdata2.obj
 0001:00001290       ??_C@_17DKNBKCHM@?$AAJ?$AAa?$AAn?$AA?$AA@ 10002290     LIBCMT:nlsdata2.obj
 0001:00001298       ??_C@_1BC@ENMNNPAJ@?$AAS?$AAa?$AAt?$AAu?$AAr?$AAd?$AAa?$AAy?$AA?$AA@ 10002298     LIBCMT:nlsdata2.obj
 0001:000012ac       ??_C@_1O@PDICJHAG@?$AAF?$AAr?$AAi?$AAd?$AAa?$AAy?$AA?$AA@ 100022ac     LIBCMT:nlsdata2.obj
 0001:000012bc       ??_C@_1BC@HHMNLIHE@?$AAT?$AAh?$AAu?$AAr?$AAs?$AAd?$AAa?$AAy?$AA?$AA@ 100022bc     LIBCMT:nlsdata2.obj
 0001:000012d0       ??_C@_1BE@EBOGMDOH@?$AAW?$AAe?$AAd?$AAn?$AAe?$AAs?$AAd?$AAa?$AAy?$AA?$AA@ 100022d0     LIBCMT:nlsdata2.obj
 0001:000012e4       ??_C@_1BA@ENFBFFEK@?$AAT?$AAu?$AAe?$AAs?$AAd?$AAa?$AAy?$AA?$AA@ 100022e4     LIBCMT:nlsdata2.obj
 0001:000012f4       ??_C@_1O@MMNBFLIA@?$AAM?$AAo?$AAn?$AAd?$AAa?$AAy?$AA?$AA@ 100022f4     LIBCMT:nlsdata2.obj
 0001:00001304       ??_C@_1O@IHNHDHPB@?$AAS?$AAu?$AAn?$AAd?$AAa?$AAy?$AA?$AA@ 10002304     LIBCMT:nlsdata2.obj
 0001:00001314       ??_C@_17GGIBDPIH@?$AAS?$AAa?$AAt?$AA?$AA@ 10002314     LIBCMT:nlsdata2.obj
 0001:0000131c       ??_C@_17HFOLPPLP@?$AAF?$AAr?$AAi?$AA?$AA@ 1000231c     LIBCMT:nlsdata2.obj
 0001:00001324       ??_C@_17PDPHAADD@?$AAT?$AAh?$AAu?$AA?$AA@ 10002324     LIBCMT:nlsdata2.obj
 0001:0000132c       ??_C@_17CJEDCEPE@?$AAW?$AAe?$AAd?$AA?$AA@ 1000232c     LIBCMT:nlsdata2.obj
 0001:00001334       ??_C@_17BMKGEGOJ@?$AAT?$AAu?$AAe?$AA?$AA@ 10002334     LIBCMT:nlsdata2.obj
 0001:0000133c       ??_C@_17KBOMKBF@?$AAM?$AAo?$AAn?$AA?$AA@ 1000233c     LIBCMT:nlsdata2.obj
 0001:00001344       ??_C@_17MBGCMIPB@?$AAS?$AAu?$AAn?$AA?$AA@ 10002344     LIBCMT:nlsdata2.obj
 0001:0000134c       ??_C@_08JCCMCCIL@HH?3mm?3ss?$AA@ 1000234c     LIBCMT:nlsdata2.obj
 0001:00001358       ??_C@_0BE@CKGJFCPC@dddd?0?5MMMM?5dd?0?5yyyy?$AA@ 10002358     LIBCMT:nlsdata2.obj
 0001:0000136c       ??_C@_08BPBNCDIB@MM?1dd?1yy?$AA@ 1000236c     LIBCMT:nlsdata2.obj
 0001:00001378       ??_C@_02CJNFDJBF@PM?$AA@   10002378     LIBCMT:nlsdata2.obj
 0001:0000137c       ??_C@_02DEDBPAFC@AM?$AA@   1000237c     LIBCMT:nlsdata2.obj
 0001:00001380       ??_C@_08EDHMEBNP@December?$AA@ 10002380     LIBCMT:nlsdata2.obj
 0001:0000138c       ??_C@_08HCHEGEOA@November?$AA@ 1000238c     LIBCMT:nlsdata2.obj
 0001:00001398       ??_C@_07JJNFCEND@October?$AA@ 10002398     LIBCMT:nlsdata2.obj
 0001:000013a0       ??_C@_09BHHEALKD@September?$AA@ 100023a0     LIBCMT:nlsdata2.obj
 0001:000013ac       ??_C@_06LBBHFDDG@August?$AA@ 100023ac     LIBCMT:nlsdata2.obj
 0001:000013b4       ??_C@_04MIEPOIFP@July?$AA@ 100023b4     LIBCMT:nlsdata2.obj
 0001:000013bc       ??_C@_04CNLMGBGM@June?$AA@ 100023bc     LIBCMT:nlsdata2.obj
 0001:000013c4       ??_C@_05DMJDNLEJ@April?$AA@ 100023c4     LIBCMT:nlsdata2.obj
 0001:000013cc       ??_C@_05HPCKOFNC@March?$AA@ 100023cc     LIBCMT:nlsdata2.obj
 0001:000013d4       ??_C@_08GNJGEPFN@February?$AA@ 100023d4     LIBCMT:nlsdata2.obj
 0001:000013e0       ??_C@_07CGJPFGJA@January?$AA@ 100023e0     LIBCMT:nlsdata2.obj
 0001:000013e8       ??_C@_03MKABNOCG@Dec?$AA@  100023e8     LIBCMT:nlsdata2.obj
 0001:000013ec       ??_C@_03JPJOFNIA@Nov?$AA@  100023ec     LIBCMT:nlsdata2.obj
 0001:000013f0       ??_C@_03BMAOKBAD@Oct?$AA@  100023f0     LIBCMT:nlsdata2.obj
 0001:000013f4       ??_C@_03GGCAPAJC@Sep?$AA@  100023f4     LIBCMT:nlsdata2.obj
 0001:000013f8       ??_C@_03IFJFEIGA@Aug?$AA@  100023f8     LIBCMT:nlsdata2.obj
 0001:000013fc       ??_C@_03LBGABGKK@Jul?$AA@  100023fc     LIBCMT:nlsdata2.obj
 0001:00001400       ??_C@_03IDFGHECI@Jun?$AA@  10002400     LIBCMT:nlsdata2.obj
 0001:00001404       ??_C@_03CNMDKL@May?$AA@    10002404     LIBCMT:nlsdata2.obj
 0001:00001408       ??_C@_03LEOLGMJP@Apr?$AA@  10002408     LIBCMT:nlsdata2.obj
 0001:0000140c       ??_C@_03ODNJBKGA@Mar?$AA@  1000240c     LIBCMT:nlsdata2.obj
 0001:00001410       ??_C@_03HJBDCHOM@Feb?$AA@  10002410     LIBCMT:nlsdata2.obj
 0001:00001414       ??_C@_03JIHJHPIE@Jan?$AA@  10002414     LIBCMT:nlsdata2.obj
 0001:00001418       ??_C@_08INBOOONO@Saturday?$AA@ 10002418     LIBCMT:nlsdata2.obj
 0001:00001424       ??_C@_06JECMNKMI@Friday?$AA@ 10002424     LIBCMT:nlsdata2.obj
 0001:0000142c       ??_C@_08HACCIKIA@Thursday?$AA@ 1000242c     LIBCMT:nlsdata2.obj
 0001:00001438       ??_C@_09DLIGFAKA@Wednesday?$AA@ 10002438     LIBCMT:nlsdata2.obj
 0001:00001444       ??_C@_07BAAGCFCM@Tuesday?$AA@ 10002444     LIBCMT:nlsdata2.obj
 0001:0000144c       ??_C@_06JLEDEDGH@Monday?$AA@ 1000244c     LIBCMT:nlsdata2.obj
 0001:00001454       ??_C@_06OOPIFAJ@Sunday?$AA@ 10002454     LIBCMT:nlsdata2.obj
 0001:0000145c       ??_C@_03FEFJNEK@Sat?$AA@   1000245c     LIBCMT:nlsdata2.obj
 0001:00001460       ??_C@_03IDIOELNC@Fri?$AA@  10002460     LIBCMT:nlsdata2.obj
 0001:00001464       ??_C@_03IOFIKPDN@Thu?$AA@  10002464     LIBCMT:nlsdata2.obj
 0001:00001468       ??_C@_03MHOMLAJA@Wed?$AA@  10002468     LIBCMT:nlsdata2.obj
 0001:0000146c       ??_C@_03NAGEINEP@Tue?$AA@  1000246c     LIBCMT:nlsdata2.obj
 0001:00001470       ??_C@_03PDAGKDH@Mon?$AA@   10002470     LIBCMT:nlsdata2.obj
 0001:00001474       ??_C@_03KOEHGMDN@Sun?$AA@  10002474     LIBCMT:nlsdata2.obj
 0001:00001478       ??_C@_1BK@DBDEIDLH@?$AAK?$AAE?$AAR?$AAN?$AAE?$AAL?$AA3?$AA2?$AA?4?$AAD?$AAL?$AAL?$AA?$AA@ 10002478     LIBCMT:tidtable.obj
 0001:00001494       ??_C@_07PEJMOBNF@FlsFree?$AA@ 10002494     LIBCMT:tidtable.obj
 0001:0000149c       ??_C@_0M@JCPCPOEF@FlsSetValue?$AA@ 1000249c     LIBCMT:tidtable.obj
 0001:000014a8       ??_C@_0M@GDNOONDI@FlsGetValue?$AA@ 100024a8     LIBCMT:tidtable.obj
 0001:000014b4       ??_C@_08KNHFBNJ@FlsAlloc?$AA@ 100024b4     LIBCMT:tidtable.obj
 0001:00001540       ??_C@_01NEMOKFLO@?$DN?$AA@ 10002540     LIBCMT:setlocal.obj
 0001:00001542       ??_C@_00CNPNBAHC@?$AA@     10002542     LIBCMT:setlocal.obj
 0001:00001548       __XcptActTab               10002548     LIBCMT:winxfltr.obj
 0001:000015d8       __First_FPE_Indx           100025d8     LIBCMT:winxfltr.obj
 0001:000015dc       __Num_FPE                  100025dc     LIBCMT:winxfltr.obj
 0001:000015e0       __XcptActTabSize           100025e0     LIBCMT:winxfltr.obj
 0001:000015e4       __XcptActTabCount          100025e4     LIBCMT:winxfltr.obj
 0001:000015e8       ??_C@_0BI@DFKBFLJE@GetProcessWindowStation?$AA@ 100025e8     LIBCMT:crtmboxw.obj
 0001:00001600       ??_C@_0BK@DEKFELLI@GetUserObjectInformationW?$AA@ 10002600     LIBCMT:crtmboxw.obj
 0001:0000161c       ??_C@_0BD@HHGDFDBJ@GetLastActivePopup?$AA@ 1000261c     LIBCMT:crtmboxw.obj
 0001:00001630       ??_C@_0BA@HNOPNCHB@GetActiveWindow?$AA@ 10002630     LIBCMT:crtmboxw.obj
 0001:00001640       ??_C@_0M@DLDCCGNP@MessageBoxW?$AA@ 10002640     LIBCMT:crtmboxw.obj
 0001:0000164c       ??_C@_1BG@GOEBHBDC@?$AAU?$AAS?$AAE?$AAR?$AA3?$AA2?$AA?4?$AAD?$AAL?$AAL?$AA?$AA@ 1000264c     LIBCMT:crtmboxw.obj
 0001:00001668       ___newctype                10002668     LIBCMT:ctype.obj
 0001:00001968       __wctype                   10002968     LIBCMT:ctype.obj
 0001:00001b70       ___newclmap                10002b70     LIBCMT:ctype.obj
 0001:00001cf0       ___newcumap                10002cf0     LIBCMT:ctype.obj
 0001:00001e78       ??_C@_0BK@CFCOFLF@?5Complete?5Object?5Locator?8?$AA@ 10002e78     LIBCMT:undname.obj
 0001:00001e94       ??_C@_0BN@MECKDCOJ@?5Class?5Hierarchy?5Descriptor?8?$AA@ 10002e94     LIBCMT:undname.obj
 0001:00001eb4       ??_C@_0BD@LGICGFMM@?5Base?5Class?5Array?8?$AA@ 10002eb4     LIBCMT:undname.obj
 0001:00001ec8       ??_C@_0BM@LDKODKLH@?5Base?5Class?5Descriptor?5at?5?$CI?$AA@ 10002ec8     LIBCMT:undname.obj
 0001:00001ee4       ??_C@_0BC@DAFEJGAK@?5Type?5Descriptor?8?$AA@ 10002ee4     LIBCMT:undname.obj
 0001:00001ef8       ??_C@_0BM@PMGGMLDN@?$GAlocal?5static?5thread?5guard?8?$AA@ 10002ef8     LIBCMT:undname.obj
 0001:00001f14       ??_C@_0CL@FGIJHLCE@?$GAmanaged?5vector?5copy?5constructor@ 10002f14     LIBCMT:undname.obj
 0001:00001f40       ??_C@_0CJ@GJELGAMM@?$GAvector?5vbase?5copy?5constructor?5i@ 10002f40     LIBCMT:undname.obj
 0001:00001f6c       ??_C@_0CD@CGAJBKEJ@?$GAvector?5copy?5constructor?5iterato@ 10002f6c     LIBCMT:undname.obj
 0001:00001f90       ??_C@_0CB@PDBIFEP@?$GAdynamic?5atexit?5destructor?5for?5?8@ 10002f90     LIBCMT:undname.obj
 0001:00001fb4       ??_C@_0BL@CLIPGLGB@?$GAdynamic?5initializer?5for?5?8?$AA@ 10002fb4     LIBCMT:undname.obj
 0001:00001fd0       ??_C@_0CM@FCBBDIGB@?$GAeh?5vector?5vbase?5copy?5constructo@ 10002fd0     LIBCMT:undname.obj
 0001:00001ffc       ??_C@_0CG@HLDDJMAG@?$GAeh?5vector?5copy?5constructor?5iter@ 10002ffc     LIBCMT:undname.obj
 0001:00002024       ??_C@_0CF@IMGKMJNO@?$GAmanaged?5vector?5destructor?5itera@ 10003024     LIBCMT:undname.obj
 0001:0000204c       ??_C@_0CG@CFDHKGGD@?$GAmanaged?5vector?5constructor?5iter@ 1000304c     LIBCMT:undname.obj
 0001:00002074       ??_C@_0BN@CKNJLHMB@?$GAplacement?5delete?$FL?$FN?5closure?8?$AA@ 10003074     LIBCMT:undname.obj
 0001:00002094       ??_C@_0BL@CNOONJFP@?$GAplacement?5delete?5closure?8?$AA@ 10003094     LIBCMT:undname.obj
 0001:000020b0       ??_C@_0P@HJKNJFNN@?$GAomni?5callsig?8?$AA@ 100030b0     LIBCMT:undname.obj
 0001:000020c0       ??_C@_09LBNFPBCA@?5delete?$FL?$FN?$AA@ 100030c0     LIBCMT:undname.obj
 0001:000020cc       ??_C@_06FHBGPFGH@?5new?$FL?$FN?$AA@ 100030cc     LIBCMT:undname.obj
 0001:000020d4       ??_C@_0CE@IIHCMGGL@?$GAlocal?5vftable?5constructor?5closu@ 100030d4     LIBCMT:undname.obj
 0001:000020f8       ??_C@_0BA@KKLDJDLB@?$GAlocal?5vftable?8?$AA@ 100030f8     LIBCMT:undname.obj
 0001:00002108       ??_C@_05KHLCHHI@?$GARTTI?$AA@ 10003108     LIBCMT:undname.obj
 0001:00002110       ??_C@_03KLGMFNMG@?$GAEH?$AA@ 10003110     LIBCMT:undname.obj
 0001:00002114       ??_C@_0BA@KBCDOMBN@?$GAudt?5returning?8?$AA@ 10003114     LIBCMT:undname.obj
 0001:00002124       ??_C@_0BL@LLKPOHJI@?$GAcopy?5constructor?5closure?8?$AA@ 10003124     LIBCMT:undname.obj
 0001:00002140       ??_C@_0CH@OOJPLCPH@?$GAeh?5vector?5vbase?5constructor?5ite@ 10003140     LIBCMT:undname.obj
 0001:00002168       ??_C@_0CA@GCEOPDGL@?$GAeh?5vector?5destructor?5iterator?8?$AA@ 10003168     LIBCMT:undname.obj
 0001:00002188       ??_C@_0CB@JONCMFFK@?$GAeh?5vector?5constructor?5iterator?8@ 10003188     LIBCMT:undname.obj
 0001:000021ac       ??_C@_0BL@NILFHHPC@?$GAvirtual?5displacement?5map?8?$AA@ 100031ac     LIBCMT:undname.obj
 0001:000021c8       ??_C@_0CE@IKBNEHA@?$GAvector?5vbase?5constructor?5iterat@ 100031c8     LIBCMT:undname.obj
 0001:000021ec       ??_C@_0BN@LFPFMEDL@?$GAvector?5destructor?5iterator?8?$AA@ 100031ec     LIBCMT:undname.obj
 0001:0000220c       ??_C@_0BO@PFGOCPJJ@?$GAvector?5constructor?5iterator?8?$AA@ 1000320c     LIBCMT:undname.obj
 0001:0000222c       ??_C@_0BN@IMDCHIKM@?$GAscalar?5deleting?5destructor?8?$AA@ 1000322c     LIBCMT:undname.obj
 0001:0000224c       ??_C@_0BO@OBMKPJIG@?$GAdefault?5constructor?5closure?8?$AA@ 1000324c     LIBCMT:undname.obj
 0001:0000226c       ??_C@_0BN@DEGPLNFK@?$GAvector?5deleting?5destructor?8?$AA@ 1000326c     LIBCMT:undname.obj
 0001:0000228c       ??_C@_0BD@JDLKDPAB@?$GAvbase?5destructor?8?$AA@ 1000328c     LIBCMT:undname.obj
 0001:000022a0       ??_C@_08OBABFOLI@?$GAstring?8?$AA@ 100032a0     LIBCMT:undname.obj
 0001:000022ac       ??_C@_0BF@KDPPACIK@?$GAlocal?5static?5guard?8?$AA@ 100032ac     LIBCMT:undname.obj
 0001:000022c4       ??_C@_08LLFFHHDJ@?$GAtypeof?8?$AA@ 100032c4     LIBCMT:undname.obj
 0001:000022d0       ??_C@_07FEEIOKP@?$GAvcall?8?$AA@ 100032d0     LIBCMT:undname.obj
 0001:000022d8       ??_C@_09BLBHBJP@?$GAvbtable?8?$AA@ 100032d8     LIBCMT:undname.obj
 0001:000022e4       ??_C@_09IFPLHPGF@?$GAvftable?8?$AA@ 100032e4     LIBCMT:undname.obj
 0001:000022f0       ??_C@_02MHEGNOJ@?$FO?$DN?$AA@ 100032f0     LIBCMT:undname.obj
 0001:000022f4       ??_C@_02DHLNPPGH@?$HM?$DN?$AA@ 100032f4     LIBCMT:undname.obj
 0001:000022f8       ??_C@_02FGJGFEAB@?$CG?$DN?$AA@ 100032f8     LIBCMT:undname.obj
 0001:000022fc       ??_C@_03CDNPDDLA@?$DM?$DM?$DN?$AA@ 100032fc     LIBCMT:undname.obj
 0001:00002300       ??_C@_03IKFCCPFF@?$DO?$DO?$DN?$AA@ 10003300     LIBCMT:undname.obj
 0001:00002304       ??_C@_02FENAOKFI@?$CF?$DN?$AA@ 10003304     LIBCMT:undname.obj
 0001:00002308       ??_C@_02FJEHGPIO@?1?$DN?$AA@ 10003308     LIBCMT:undname.obj
 0001:0000230c       ??_C@_02FKMDLLOA@?9?$DN?$AA@ 1000330c     LIBCMT:undname.obj
 0001:00002310       ??_C@_02FOEOMHFC@?$CL?$DN?$AA@ 10003310     LIBCMT:undname.obj
 0001:00002314       ??_C@_02FPIMKNGF@?$CK?$DN?$AA@ 10003314     LIBCMT:undname.obj
 0001:00002318       ??_C@_02NONPIBCD@?$HM?$HM?$AA@ 10003318     LIBCMT:undname.obj
 0001:0000231c       ??_C@_02PPKAJPJL@?$CG?$CG?$AA@ 1000331c     LIBCMT:undname.obj
 0001:00002320       ??_C@_01DNKMNLPK@?$HM?$AA@ 10003320     LIBCMT:undname.obj
 0001:00002324       ??_C@_01JKBOJNNK@?$FO?$AA@ 10003324     LIBCMT:undname.obj
 0001:00002328       ??_C@_01PJKLJHI@?$HO?$AA@  10003328     LIBCMT:undname.obj
 0001:0000232c       ??_C@_02HCKGKOFO@?$CI?$CJ?$AA@ 1000332c     LIBCMT:undname.obj
 0001:00002330       ??_C@_01IHBHIGKO@?0?$AA@   10003330     LIBCMT:undname.obj
 0001:00002334       ??_C@_02EEKDKGMJ@?$DO?$DN?$AA@ 10003334     LIBCMT:undname.obj
 0001:00002338       ??_C@_01PPODPGHN@?$DO?$AA@ 10003338     LIBCMT:undname.obj
 0001:0000233c       ??_C@_02EHCHHCKH@?$DM?$DN?$AA@ 1000333c     LIBCMT:undname.obj
 0001:00002340       ??_C@_01MNNFJEPP@?$DM?$AA@ 10003340     LIBCMT:undname.obj
 0001:00002344       ??_C@_01FGNFDNOH@?$CF?$AA@ 10003344     LIBCMT:undname.obj
 0001:00002348       ??_C@_01KMDKNFGN@?1?$AA@   10003348     LIBCMT:undname.obj
 0001:0000234c       ??_C@_03MNHNFDLC@?9?$DO?$CK?$AA@ 1000334c     LIBCMT:undname.obj
 0001:00002350       ??_C@_01HNPIGOCE@?$CG?$AA@ 10003350     LIBCMT:undname.obj
 0001:00002354       ??_C@_01MIFGBAGJ@?$CL?$AA@ 10003354     LIBCMT:undname.obj
 0001:00002358       ??_C@_01JOAMLHOP@?9?$AA@   10003358     LIBCMT:undname.obj
 0001:0000235c       ??_C@_02BAABKJLB@?9?9?$AA@ 1000335c     LIBCMT:undname.obj
 0001:00002360       ??_C@_02ECNGHCIF@?$CL?$CL?$AA@ 10003360     LIBCMT:undname.obj
 0001:00002364       ??_C@_01NBENCBCI@?$CK?$AA@ 10003364     LIBCMT:undname.obj
 0001:00002368       ??_C@_02HBOOOICD@?9?$DO?$AA@ 10003368     LIBCMT:undname.obj
 0001:0000236c       ??_C@_08LHJFAFGD@operator?$AA@ 1000336c     LIBCMT:undname.obj
 0001:00002378       ??_C@_02GPECMEKF@?$FL?$FN?$AA@ 10003378     LIBCMT:undname.obj
 0001:0000237c       ??_C@_02FDNJECIE@?$CB?$DN?$AA@ 1000337c     LIBCMT:undname.obj
 0001:00002380       ??_C@_02EGOFBIJA@?$DN?$DN?$AA@ 10003380     LIBCMT:undname.obj
 0001:00002384       ??_C@_01DCLJPIOD@?$CB?$AA@ 10003384     LIBCMT:undname.obj
 0001:00002388       ??_C@_02FODMEDOG@?$DM?$DM?$AA@ 10003388     LIBCMT:undname.obj
 0001:0000238c       ??_C@_02GPIOPFAK@?$DO?$DO?$AA@ 1000338c     LIBCMT:undname.obj
 0001:00002390       ??_C@_07FPCDHGMM@?5delete?$AA@ 10003390     LIBCMT:undname.obj
 0001:00002398       ??_C@_04NIHEBCM@?5new?$AA@ 10003398     LIBCMT:undname.obj
 0001:000023a0       ??_C@_0M@GFIIJFMG@__unaligned?$AA@ 100033a0     LIBCMT:undname.obj
 0001:000023ac       ??_C@_0L@PILCLIHE@__restrict?$AA@ 100033ac     LIBCMT:undname.obj
 0001:000023b8       ??_C@_07JOMMBBKO@__ptr64?$AA@ 100033b8     LIBCMT:undname.obj
 0001:000023c0       ??_C@_06GHPCKEAG@__eabi?$AA@ 100033c0     LIBCMT:undname.obj
 0001:000023c8       ??_C@_09HIJEGCPM@__clrcall?$AA@ 100033c8     LIBCMT:undname.obj
 0001:000023d4       ??_C@_0L@JMKHOMEK@__fastcall?$AA@ 100033d4     LIBCMT:undname.obj
 0001:000023e0       ??_C@_0L@NPHFGOKO@__thiscall?$AA@ 100033e0     LIBCMT:undname.obj
 0001:000023ec       ??_C@_09IFJBGAPI@__stdcall?$AA@ 100033ec     LIBCMT:undname.obj
 0001:000023f8       ??_C@_08GHMPAG@__pascal?$AA@ 100033f8     LIBCMT:undname.obj
 0001:00002404       ??_C@_07KOLFKCDI@__cdecl?$AA@ 10003404     LIBCMT:undname.obj
 0001:0000240c       ??_C@_08EHJDFFNH@__based?$CI?$AA@ 1000340c     LIBCMT:undname.obj
 0001:000025a0       __load_config_used         100035a0     LIBCMT:loadcfg.obj
 0001:000025e8       ??_R4bad_alloc@std@@6B@    100035e8     LIBCMT:new.obj
 0001:000025fc       ??_R3bad_alloc@std@@8      100035fc     LIBCMT:new.obj
 0001:0000260c       ??_R2bad_alloc@std@@8      1000360c     LIBCMT:new.obj
 0001:00002618       ??_R1A@?0A@EA@bad_alloc@std@@8 10003618     LIBCMT:new.obj
 0001:00002634       ??_R1A@?0A@EA@exception@std@@8 10003634     LIBCMT:new.obj
 0001:00002650       ??_R3exception@std@@8      10003650     LIBCMT:new.obj
 0001:00002660       ??_R2exception@std@@8      10003660     LIBCMT:new.obj
 0001:00002668       ??_R4exception@std@@6B@    10003668     LIBCMT:stdexcpt.obj
 0001:0000267c       ??_R4type_info@@6B@        1000367c     LIBCMT:typinfo.obj
 0001:00002690       ??_R3type_info@@8          10003690     LIBCMT:typinfo.obj
 0001:000026a0       ??_R2type_info@@8          100036a0     LIBCMT:typinfo.obj
 0001:000026a8       ??_R1A@?0A@EA@type_info@@8 100036a8     LIBCMT:typinfo.obj
 0001:000026d0       ___safe_se_handler_table   100036d0     <linker-defined>
 0001:000026dc       ___rtc_iaa                 100036dc     LIBCMT:_initsect_.obj
 0001:000026e0       ___rtc_izz                 100036e0     LIBCMT:_initsect_.obj
 0001:000026e4       ___rtc_taa                 100036e4     LIBCMT:_initsect_.obj
 0001:000026e8       ___rtc_tzz                 100036e8     LIBCMT:_initsect_.obj
 0001:000026f0       __alloca_probe             100036f0     chkstk.obj
 0001:000026f0       __chkstk                   100036f0 f   chkstk.obj
 0001:00002720       ?GetLangString@PluginDialogBuilder@@MAEPB_WH@Z 10003720 f i FARCmds.obj
 0001:00002740       _GetGlobalInfoW@4          10003740 f   FARCmds.obj
 0001:000027c0       _SetStartupInfoW@4         100037c0 f   FARCmds.obj
 0001:00002a20       _OpenW@4                   10003a20 f   FARCmds.obj
 0001:00002cb0       _GetPluginInfoW@4          10003cb0 f   FARCmds.obj
 0001:00002d00       ?SaveValue@?$DialogItemBinding@UFarDialogItem@@@@UAEXPAUFarDialogItem@@H@Z 10003d00 f i FARCmds.obj
 0001:00002d00       ?InitDialogItem@?$DialogBuilderBase@UFarDialogItem@@@@MAEXPAUFarDialogItem@@PB_W@Z 10003d00 f i FARCmds.obj
 0001:00002d10       ?TextWidth@?$DialogBuilderBase@UFarDialogItem@@@@MAEHABUFarDialogItem@@@Z 10003d10 f i FARCmds.obj
 0001:00002d20       ?DoShowDialog@?$DialogBuilderBase@UFarDialogItem@@@@MAEHXZ 10003d20 f i FARCmds.obj
 0001:00002d30       ?GetLangString@?$DialogBuilderBase@UFarDialogItem@@@@MAEPB_WH@Z 10003d30 f i FARCmds.obj
 0001:00002d30       ?CreateRadioButtonBinding@?$DialogBuilderBase@UFarDialogItem@@@@MAEPAU?$DialogItemBinding@UFarDialogItem@@@@PAH@Z 10003d30 f i FARCmds.obj
 0001:00002d40       ??1?$DialogBuilderBase@UFarDialogItem@@@@MAE@XZ 10003d40 f i FARCmds.obj
 0001:00002d90       ?AddIntEditField@?$DialogBuilderBase@UFarDialogItem@@@@UAEPAUFarDialogItem@@PAHH@Z 10003d90 f i FARCmds.obj
 0001:00002d90       ?CreateCheckBoxBinding@?$DialogBuilderBase@UFarDialogItem@@@@MAEPAU?$DialogItemBinding@UFarDialogItem@@@@PAHH@Z 10003d90 f i FARCmds.obj
 0001:00002d90       ?AddUIntEditField@?$DialogBuilderBase@UFarDialogItem@@@@UAEPAUFarDialogItem@@PAIH@Z 10003d90 f i FARCmds.obj
 0001:00002da0       ??_E?$DialogBuilderBase@UFarDialogItem@@@@MAEPAXI@Z 10003da0 f i FARCmds.obj
 0001:00002da0       ??_G?$DialogBuilderBase@UFarDialogItem@@@@MAEPAXI@Z 10003da0 f i FARCmds.obj
 0001:00002dc0       ?ReallocDialogItems@?$DialogBuilderBase@UFarDialogItem@@@@IAEXXZ 10003dc0 f i FARCmds.obj
 0001:00002e90       ?UpdateSecondColumnPosition@?$DialogBuilderBase@UFarDialogItem@@@@IAEXXZ 10003e90 f i FARCmds.obj
 0001:00002ef0       ?SaveValues@?$DialogBuilderBase@UFarDialogItem@@@@IAEXXZ 10003ef0 f i FARCmds.obj
 0001:00002f40       ?MaxTextWidth@?$DialogBuilderBase@UFarDialogItem@@@@IAEHXZ 10003f40 f i FARCmds.obj
 0001:00003000       ??0PluginUIntEditFieldBinding@@QAE@ABUPluginStartupInfo@@PAPAXHPAIH@Z 10004000 f i FARCmds.obj
 0001:000030a0       ?SaveValue@PluginUIntEditFieldBinding@@UAEXPAUFarDialogItem@@H@Z 100040a0 f i FARCmds.obj
 0001:000030d0       ?InitDialogItem@PluginDialogBuilder@@MAEXPAUFarDialogItem@@PB_W@Z 100040d0 f i FARCmds.obj
 0001:000030f0       ?TextWidth@PluginDialogBuilder@@MAEHABUFarDialogItem@@@Z 100040f0 f i FARCmds.obj
 0001:00003110       ?DoShowDialog@PluginDialogBuilder@@MAEHXZ 10004110 f i FARCmds.obj
 0001:00003170       ?SaveValue@PluginCheckBoxBinding@@UAEXPAUFarDialogItem@@H@Z 10004170 f i FARCmds.obj
 0001:000031b0       ?SaveValue@PluginRadioButtonBinding@@UAEXPAUFarDialogItem@@H@Z 100041b0 f i FARCmds.obj
 0001:000031e0       ??0PluginIntEditFieldBinding@@QAE@ABUPluginStartupInfo@@PAPAXHPAHH@Z 100041e0 f i FARCmds.obj
 0001:00003280       ?SaveValue@PluginIntEditFieldBinding@@UAEXPAUFarDialogItem@@H@Z 10004280 f i FARCmds.obj
 0001:000032b0       ?CreateCheckBoxBinding@PluginDialogBuilder@@MAEPAU?$DialogItemBinding@UFarDialogItem@@@@PAHH@Z 100042b0 f i FARCmds.obj
 0001:00003300       ?CreateRadioButtonBinding@PluginDialogBuilder@@MAEPAU?$DialogItemBinding@UFarDialogItem@@@@PAH@Z 10004300 f i FARCmds.obj
 0001:00003350       ??_GPluginDialogBuilder@@UAEPAXI@Z 10004350 f i FARCmds.obj
 0001:00003350       ??_EPluginDialogBuilder@@UAEPAXI@Z 10004350 f i FARCmds.obj
 0001:00003390       ?AddCheckbox@?$DialogBuilderBase@UFarDialogItem@@@@QAEPAUFarDialogItem@@HPAHH_N@Z 10004390 f i FARCmds.obj
 0001:000034c0       ?AddRadioButtons@?$DialogBuilderBase@UFarDialogItem@@@@QAEXPAHHQBH_N@Z 100044c0 f i FARCmds.obj
 0001:00003620       ?AddTextBefore@?$DialogBuilderBase@UFarDialogItem@@@@QAEPAUFarDialogItem@@PAU2@H@Z 10004620 f i FARCmds.obj
 0001:00003750       ?AddSeparator@?$DialogBuilderBase@UFarDialogItem@@@@QAEXPB_W@Z 10004750 f i FARCmds.obj
 0001:000037c0       ?AddButtons@?$DialogBuilderBase@UFarDialogItem@@@@QAEXHPBHHH@Z 100047c0 f i FARCmds.obj
 0001:00003920       ?UpdateBorderSize@?$DialogBuilderBase@UFarDialogItem@@@@IAEXXZ 10004920 f i FARCmds.obj
 0001:000039d0       ??_G?$DialogItemBinding@UFarDialogItem@@@@UAEPAXI@Z 100049d0 f i FARCmds.obj
 0001:000039d0       ??_GPluginRadioButtonBinding@@UAEPAXI@Z 100049d0 f i FARCmds.obj
 0001:000039d0       ??_EPluginIntEditFieldBinding@@UAEPAXI@Z 100049d0 f i FARCmds.obj
 0001:000039d0       ??_GPluginIntEditFieldBinding@@UAEPAXI@Z 100049d0 f i FARCmds.obj
 0001:000039d0       ??_E?$DialogItemBinding@UFarDialogItem@@@@UAEPAXI@Z 100049d0 f i FARCmds.obj
 0001:000039d0       ??_GPluginCheckBoxBinding@@UAEPAXI@Z 100049d0 f i FARCmds.obj
 0001:000039d0       ??_EPluginRadioButtonBinding@@UAEPAXI@Z 100049d0 f i FARCmds.obj
 0001:000039d0       ??_GPluginUIntEditFieldBinding@@UAEPAXI@Z 100049d0 f i FARCmds.obj
 0001:000039d0       ??_EPluginUIntEditFieldBinding@@UAEPAXI@Z 100049d0 f i FARCmds.obj
 0001:000039d0       ??_EPluginCheckBoxBinding@@UAEPAXI@Z 100049d0 f i FARCmds.obj
 0001:000039f0       ??0PluginDialogBuilder@@QAE@ABUPluginStartupInfo@@ABU_GUID@@1HPB_WP6GHPAXHH3@Z3_K@Z 100049f0 f i FARCmds.obj
 0001:00003b00       ?AddIntEditField@PluginDialogBuilder@@UAEPAUFarDialogItem@@PAHH@Z 10004b00 f i FARCmds.obj
 0001:00003bc0       ?AddUIntEditField@PluginDialogBuilder@@UAEPAUFarDialogItem@@PAIH@Z 10004bc0 f i FARCmds.obj
 0001:00003c80       _ConfigureW@4              10004c80 f   FARCmds.obj
 0001:00004010       ?GetMsg@@YAPB_WH@Z         10005010 f   Mix.obj
 0001:00004030       ?ExpandEnv@@YAPA_WPB_WPAK@Z 10005030 f   Mix.obj
 0001:00004090       ?GetInt@@YAHPB_WPA_W@Z     10005090 f   Mix.obj
 0001:00004170       ?ReplaceStrings@@YAHPA_WPB_W1HH@Z 10005170 f   Mix.obj
 0001:000042f0       ?PartCmdLine@@YAHPB_WPAPA_W1@Z 100052f0 f   Mix.obj
 0001:00004580       ?ProcessOSAliases@@YAPA_WPB_W@Z 10005580 f   Mix.obj
 0001:000047a0       ?GetShellLinkPath@@YAPA_WPB_W@Z 100057a0 f   Mix.obj
 0001:00004a20       ?StrToGuid@@YA_NPB_WPAU_GUID@@@Z 10005a20 f   Mix.obj
 0001:00004a40       ?IsTextUTF8@@YA_NPBDI@Z    10005a40 f   Mix.obj
 0001:00004ab0       ?GetCPBuffer@@YAIPBXIPAI@Z 10005ab0 f   Mix.obj
 0001:00004b80       ?ConvertBuffer@@YAPA_WPA_WIHAAIPA_N@Z 10005b80 f   Mix.obj
 0001:00004ca0       ??0ConsoleTitle@@QAE@PB_W@Z 10005ca0 f i OpenCmd.obj
 0001:00004d10       ??1ConsoleTitle@@QAE@XZ    10005d10 f i OpenCmd.obj
 0001:00004d30       ??0MakeVETitle@@QAE@PB_W0@Z 10005d30 f i OpenCmd.obj
 0001:00004f40       ?isDevice@@YA_NPB_W0@Z     10005f40 f i OpenCmd.obj
 0001:00005270       ?ThreadWhatUpdateScreen@@YGKPAX@Z 10006270 f   OpenCmd.obj
 0001:000058b0       ?__proc_Load@@YAPA_WHPA_W@Z 100068b0 f   OpenCmd.obj
 0001:00005910       ?__proc_Unload@@YAPA_WHPA_W@Z 10006910 f   OpenCmd.obj
 0001:00005a00       ?__proc_Goto@@YAPA_WHPA_W@Z 10006a00 f   OpenCmd.obj
 0001:00005a60       ?__proc_WhereIs@@YAPA_WHPA_W_N@Z 10006a60 f   OpenCmd.obj
 0001:00005f70       ?__proc_Link@@YA_NHPA_W@Z  10006f70 f   OpenCmd.obj
 0001:00006450       ?OpenFromCommandLine@@YAPA_WPB_W@Z 10007450 f   OpenCmd.obj
 0001:00007230       _memcpy                    10008230 f   LIBCMT:memcpy.obj
 0001:00007591       _free                      10008591 f   LIBCMT:free.obj
 0001:000075cb       _malloc                    100085cb f   LIBCMT:malloc.obj
 0001:0000765f       ??3@YAXPAX@Z               1000865f f   LIBCMT:delete.obj
 0001:0000766a       ??1bad_alloc@std@@UAE@XZ   1000866a f i LIBCMT:new.obj
 0001:00007675       ??_Ebad_alloc@std@@UAEPAXI@Z 10008675 f i LIBCMT:new.obj
 0001:00007675       ??_Gbad_alloc@std@@UAEPAXI@Z 10008675 f i LIBCMT:new.obj
 0001:0000769c       ??0bad_alloc@std@@QAE@ABV01@@Z 1000869c f i LIBCMT:new.obj
 0001:000076b9       ??2@YAPAXI@Z               100086b9 f   LIBCMT:new.obj
 0001:00007740       _memset                    10008740 f   LIBCMT:memset.obj
 0001:000077ba       _wcschr                    100087ba f   LIBCMT:wcschr.obj
 0001:000077e1       _wcsstr                    100087e1 f   LIBCMT:wcsstr.obj
 0001:00007850       _memmove                   10008850 f   LIBCMT:memmove.obj
 0001:00007bb1       ??0_LocaleUpdate@@QAE@PAUlocaleinfo_struct@@@Z 10008bb1 f i LIBCMT:memicmp.obj
 0001:00007c38       __memicmp_l                10008c38 f   LIBCMT:memicmp.obj
 0001:00007d03       __memicmp                  10008d03 f   LIBCMT:memicmp.obj
 0001:00007d57       _realloc                   10008d57 f   LIBCMT:realloc.obj
 0001:00007e04       _wcsncmp                   10008e04 f   LIBCMT:wcsncmp.obj
 0001:00007e3d       __CRT_INIT@12              10008e3d f   LIBCMT:dllcrt0.obj
 0001:00008097       __DllMainCRTStartup@12     10009097 f   LIBCMT:dllcrt0.obj
 0001:000080ba       __VEC_memcpy               100090ba f   LIBCMT:p4_memcpy.obj
 0001:000081bd       ___sse2_available_init     100091bd f   LIBCMT:cpu_disp.obj
 0001:000081cd       __get_errno_from_oserr     100091cd f   LIBCMT:dosmap.obj
 0001:0000820f       __errno                    1000920f f   LIBCMT:dosmap.obj
 0001:00008222       __heap_init                10009222 f   LIBCMT:heapinit.obj
 0001:00008240       __heap_term                10009240 f   LIBCMT:heapinit.obj
 0001:00008254       ___crtCorExitProcess       10009254 f   LIBCMT:crt0dat.obj
 0001:0000827f       ___crtExitProcess          1000927f f   LIBCMT:crt0dat.obj
 0001:00008297       __lockexit                 10009297 f   LIBCMT:crt0dat.obj
 0001:000082a0       __unlockexit               100092a0 f   LIBCMT:crt0dat.obj
 0001:000082a9       __init_pointers            100092a9 f   LIBCMT:crt0dat.obj
 0001:000082dc       __initterm_e               100092dc f   LIBCMT:crt0dat.obj
 0001:00008300       __cinit                    10009300 f   LIBCMT:crt0dat.obj
 0001:000084d7       __exit                     100094d7 f   LIBCMT:crt0dat.obj
 0001:000084ed       __cexit                    100094ed f   LIBCMT:crt0dat.obj
 0001:000084fc       __amsg_exit                100094fc f   LIBCMT:crt0dat.obj
 0001:0000851a       __GET_RTERRMSG             1000951a f   LIBCMT:crt0msg.obj
 0001:00008540       __NMSG_WRITE               10009540 f   LIBCMT:crt0msg.obj
 0001:000086ef       __FF_MSGBANNER             100096ef f   LIBCMT:crt0msg.obj
 0001:00008728       __initp_heap_handler       10009728 f   LIBCMT:handler.obj
 0001:00008737       __callnewh                 10009737 f   LIBCMT:handler.obj
 0001:0000875f       ??0exception@std@@QAE@ABQBDH@Z 1000975f f   LIBCMT:stdexcpt.obj
 0001:0000877c       ?what@exception@std@@UBEPBDXZ 1000977c f   LIBCMT:stdexcpt.obj
 0001:00008789       ?_Copy_str@exception@std@@AAEXPBD@Z 10009789 f   LIBCMT:stdexcpt.obj
 0001:000087c9       ?_Tidy@exception@std@@AAEXXZ 100097c9 f   LIBCMT:stdexcpt.obj
 0001:000087e7       ??4exception@std@@QAEAAV01@ABV01@@Z 100097e7 f   LIBCMT:stdexcpt.obj
 0001:0000881c       ??1exception@std@@UAE@XZ   1000981c f   LIBCMT:stdexcpt.obj
 0001:00008827       ??_Gexception@std@@UAEPAXI@Z 10009827 f i LIBCMT:stdexcpt.obj
 0001:00008827       ??_Eexception@std@@UAEPAXI@Z 10009827 f i LIBCMT:stdexcpt.obj
 0001:0000884e       ??0exception@std@@QAE@ABV01@@Z 1000984e f   LIBCMT:stdexcpt.obj
 0001:00008873       ??1type_info@@UAE@XZ       10009873 f   LIBCMT:typinfo.obj
 0001:00008883       ??_Etype_info@@UAEPAXI@Z   10009883 f i LIBCMT:typinfo.obj
 0001:00008883       ??_Gtype_info@@UAEPAXI@Z   10009883 f i LIBCMT:typinfo.obj
 0001:0000895a       ___onexitinit              1000995a f   LIBCMT:onexit.obj
 0001:0000898b       __onexit                   1000998b f   LIBCMT:onexit.obj
 0001:000089c7       _atexit                    100099c7 f   LIBCMT:onexit.obj
 0001:000089de       __CxxThrowException@8      100099de f   LIBCMT:throw.obj
 0001:00008a2a       __VEC_memzero              10009a2a f   LIBCMT:p4_memset.obj
 0001:00008d07       ___updatetmbcinfo          10009d07 f   LIBCMT:mbctype.obj
 0001:00008e27       __setmbcp_nolock           10009e27 f   LIBCMT:mbctype.obj
 0001:00009010       __setmbcp                  1000a010 f   LIBCMT:mbctype.obj
 0001:000091aa       ___initmbctable            1000a1aa f   LIBCMT:mbctype.obj
 0001:000091c8       ___addlocaleref            1000a1c8 f   LIBCMT:localref.obj
 0001:00009257       ___removelocaleref         1000a257 f   LIBCMT:localref.obj
 0001:000092f0       ___freetlocinfo            1000a2f0 f   LIBCMT:localref.obj
 0001:0000943b       __updatetlocinfoEx_nolock  1000a43b f   LIBCMT:localref.obj
 0001:00009488       ___updatetlocinfo          1000a488 f   LIBCMT:localref.obj
 0001:00009501       __encoded_null             1000a501 f   LIBCMT:tidtable.obj
 0001:0000950a       ___crtTlsAlloc@4           1000a50a f   LIBCMT:tidtable.obj
 0001:00009513       ___set_flsgetvalue         1000a513 f   LIBCMT:tidtable.obj
 0001:00009547       __mtterm                   1000a547 f   LIBCMT:tidtable.obj
 0001:00009584       __initptd                  1000a584 f   LIBCMT:tidtable.obj
 0001:00009638       __getptd_noexit            1000a638 f   LIBCMT:tidtable.obj
 0001:000096b1       __getptd                   1000a6b1 f   LIBCMT:tidtable.obj
 0001:000096cb       __freefls@4                1000a6cb f   LIBCMT:tidtable.obj
 0001:000097fa       __freeptd                  1000a7fa f   LIBCMT:tidtable.obj
 0001:00009868       __mtinit                   1000a868 f   LIBCMT:tidtable.obj
 0001:000099e3       __tolower_l                1000a9e3 f   LIBCMT:tolower.obj
 0001:00009b00       ___ascii_memicmp           1000ab00 f   LIBCMT:_memicmp.obj
 0001:00009b59       __initp_misc_invarg        1000ab59 f   LIBCMT:invarg.obj
 0001:00009b68       __call_reportfault         1000ab68 f   LIBCMT:invarg.obj
 0001:00009c91       __invoke_watson            1000ac91 f   LIBCMT:invarg.obj
 0001:00009cb6       __invalid_parameter        1000acb6 f   LIBCMT:invarg.obj
 0001:00009ce3       __invalid_parameter_noinfo 1000ace3 f   LIBCMT:invarg.obj
 0001:00009cf3       __malloc_crt               1000acf3 f   LIBCMT:crtheap.obj
 0001:00009d38       __calloc_crt               1000ad38 f   LIBCMT:crtheap.obj
 0001:00009d84       __realloc_crt              1000ad84 f   LIBCMT:crtheap.obj
 0001:00009dd2       __ioinit                   1000add2 f   LIBCMT:ioinit.obj
 0001:0000a017       __ioterm                   1000b017 f   LIBCMT:ioinit.obj
 0001:0000a06a       __setenvp                  1000b06a f   LIBCMT:stdenvp.obj
 0001:0000a2e0       __setargv                  1000b2e0 f   LIBCMT:stdargv.obj
 0001:0000a39b       ___crtGetEnvironmentStringsA 1000b39b f   LIBCMT:a_env.obj
 0001:0000a432       __RTC_Initialize           1000b432 f   LIBCMT:_initsect_.obj
 0001:0000a458       __RTC_Terminate            1000b458 f   LIBCMT:_initsect_.obj
 0001:0000a480       __SEH_prolog4              1000b480 f   LIBCMT:sehprolg4.obj
 0001:0000a4c5       __SEH_epilog4              1000b4c5 f   LIBCMT:sehprolg4.obj
 0001:0000a4e0       __except_handler4          1000b4e0 f   LIBCMT:chandler4.obj
 0001:0000a66f       __XcptFilter               1000b66f f   LIBCMT:winxfltr.obj
 0001:0000a7b9       ___CppXcptFilter           1000b7b9 f   LIBCMT:winxfltr.obj
 0001:0000a7d9       _DllMain@12                1000b7d9 f   LIBCMT:dllmain.obj
 0001:0000a7df       ___security_init_cookie    1000b7df f   LIBCMT:gs_support.obj
 0001:0000a87a       __mtinitlocks              1000b87a f   LIBCMT:mlock.obj
 0001:0000a8c4       __mtdeletelocks            1000b8c4 f   LIBCMT:mlock.obj
 0001:0000a91b       __unlock                   1000b91b f   LIBCMT:mlock.obj
 0001:0000a932       __mtinitlocknum            1000b932 f   LIBCMT:mlock.obj
 0001:0000a9f4       __lock                     1000b9f4 f   LIBCMT:mlock.obj
 0001:0000aa27       ?terminate@@YAXXZ          1000ba27 f   LIBCMT:hooks.obj
 0001:0000aa60       __initp_eh_hooks           1000ba60 f   LIBCMT:hooks.obj
 0001:0000aa71       __initp_misc_winsig        1000ba71 f   LIBCMT:winsig.obj
 0001:0000aac6       ___get_sigabrt             1000bac6 f   LIBCMT:winsig.obj
 0001:0000aad3       _raise                     1000bad3 f   LIBCMT:winsig.obj
 0001:0000ac76       __initp_misc_rand_s        1000bc76 f   LIBCMT:rand_s.obj
 0001:0000ac85       __initp_misc_purevirt      1000bc85 f   LIBCMT:inithelp.obj
 0001:0000ac94       __initp_misc_cfltcvt_tab   1000bc94 f   LIBCMT:cmiscdat.obj
 0001:0000acc0       __ValidateImageBase        1000bcc0 f   LIBCMT:pesect.obj
 0001:0000ad00       __FindPESection            1000bd00 f   LIBCMT:pesect.obj
 0001:0000ad50       __IsNonwritableInCurrentImage 1000bd50 f   LIBCMT:pesect.obj
 0001:0000ae10       _strlen                    1000be10 f   LIBCMT:strlen.obj
 0001:0000ae9b       ___crtMessageBoxW          1000be9b f   LIBCMT:crtmboxw.obj
 0001:0000b007       _wcscat_s                  1000c007 f   LIBCMT:wcscat_s.obj
 0001:0000b07c       _wcsncpy_s                 1000c07c f   LIBCMT:wcsncpy_s.obj
 0001:0000b149       _wcslen                    1000c149 f   LIBCMT:wcslen.obj
 0001:0000b164       _wcscpy_s                  1000c164 f   LIBCMT:wcscpy_s.obj
 0001:0000b1c7       __set_error_mode           1000c1c7 f   LIBCMT:errmode.obj
 0001:0000b206       @__security_check_cookie@4 1000c206 f   LIBCMT:secchk.obj
 0001:0000b215       _strcpy_s                  1000c215 f   LIBCMT:strcpy_s.obj
 0001:0000b274       ?_Type_info_dtor@type_info@@CAXPAV1@@Z 1000c274 f   LIBCMT:typname.obj
 0001:0000b2f0       _strcmp                    1000c2f0 f   LIBCMT:strcmp.obj
 0001:0000b378       __msize                    1000c378 f   LIBCMT:msize.obj
 0001:0000b3ab       __freea                    1000c3ab f i LIBCMT:a_map.obj
 0001:0000b5b2       ___crtLCMapStringA         1000c5b2 f   LIBCMT:a_map.obj
 0001:0000b6df       ___crtGetStringTypeA       1000c6df f   LIBCMT:a_str.obj
 0001:0000b71f       ___free_lc_time            1000c71f f   LIBCMT:inittime.obj
 0001:0000ba96       ___free_lconv_num          1000ca96 f   LIBCMT:initnum.obj
 0001:0000baff       ___free_lconv_mon          1000caff f   LIBCMT:initmon.obj
 0001:0000bbfd       __isleadbyte_l             1000cbfd f i LIBCMT:_wctype.obj
 0001:0000bc35       __isctype_l                1000cc35 f   LIBCMT:isctype.obj
 0001:0000bced       __crt_debugger_hook        1000cced f   LIBCMT:dbghook.obj
 0001:0000bd00       _strcspn                   1000cd00 f   LIBCMT:strcspn.obj
 0001:0000bd50       _strpbrk                   1000cd50 f   LIBCMT:strpbrk.obj
 0001:0000bd90       __calloc_impl              1000cd90 f   LIBCMT:calloc_impl.obj
 0001:0000be65       __ismbblead                1000ce65 f   LIBCMT:ismbbyte.obj
 0001:0000be80       __local_unwind4            1000ce80 f   LIBCMT:exsup4.obj
 0001:0000bf56       __seh_longjmp_unwind4@4    1000cf56 f   LIBCMT:exsup4.obj
 0001:0000bf72       @_EH4_CallFilterFunc@8     1000cf72 f   LIBCMT:exsup4.obj
 0001:0000bf89       @_EH4_TransferToHandler@8  1000cf89 f   LIBCMT:exsup4.obj
 0001:0000bfa2       @_EH4_GlobalUnwind2@8      1000cfa2 f   LIBCMT:exsup4.obj
 0001:0000bfbb       @_EH4_LocalUnwind@16       1000cfbb f   LIBCMT:exsup4.obj
 0001:0000bfd2       _abort                     1000cfd2 f   LIBCMT:abort.obj
 0001:0000c005       __fptrap                   1000d005 f   LIBCMT:crt0fp.obj
 0001:0000c00e       ___report_gsfailure        1000d00e f   LIBCMT:gs_report.obj
 0001:0000c120       __alloca_probe_16          1000d120 f   LIBCMT:alloca16.obj
 0001:0000c136       __alloca_probe_8           1000d136     LIBCMT:alloca16.obj
 0001:0000c150       __global_unwind2           1000d150 f   LIBCMT:exsup.obj
 0001:0000c1b5       __local_unwind2            1000d1b5 f   LIBCMT:exsup.obj
 0001:0000c239       __abnormal_termination     1000d239 f   LIBCMT:exsup.obj
 0001:0000c25c       __NLG_Notify1              1000d25c f   LIBCMT:exsup.obj
 0001:0000c265       __NLG_Notify               1000d265 f   LIBCMT:exsup.obj
 0001:0000c27c       __NLG_Dispatch             1000d27c     LIBCMT:exsup.obj
 0001:0000c27c       __NLG_Dispatch2            1000d27c     LIBCMT:exsup.obj
 0001:0000c284       __NLG_Call                 1000d284 f   LIBCMT:exsup.obj
 0001:0000c286       __NLG_Return2              1000d286     LIBCMT:exsup.obj
 0001:0000c290       __aulldvrm                 1000d290 f   LIBCMT:ulldvrm.obj
 0001:0000c330       ___ascii_strnicmp          1000d330 f   LIBCMT:_strnicm.obj
 0001:0000c3a0       __allmul                   1000d3a0 f   LIBCMT:llmul.obj
 0001:0000c3d4       _RtlUnwind@16              1000d3d4 f   kernel32:KERNEL32.dll
 0001:0000c3da       __swab                     1000d3da f   LIBCMT:swab.obj
 0001:0000c3da       _swab                      1000d3da f   LIBCMT:swab.obj
 0001:0000c440       __TI2?AVbad_alloc@std@@    1000d440     LIBCMT:new.obj
 0001:0000c450       __CTA2?AVbad_alloc@std@@   1000d450     LIBCMT:new.obj
 0001:0000c45c       __CT??_R0?AVbad_alloc@std@@@8??0bad_alloc@std@@QAE@ABV01@@Z12 1000d45c     LIBCMT:new.obj
 0001:0000c478       __CT??_R0?AVexception@std@@@8??0exception@std@@QAE@ABV01@@Z12 1000d478     LIBCMT:new.obj
 0001:0000c664       __IMPORT_DESCRIPTOR_KERNEL32 1000d664     kernel32:KERNEL32.dll
 0001:0000c678       __IMPORT_DESCRIPTOR_USER32 1000d678     user32:USER32.dll
 0001:0000c68c       __IMPORT_DESCRIPTOR_ADVAPI32 1000d68c     advapi32:ADVAPI32.dll
 0001:0000c6a0       __IMPORT_DESCRIPTOR_ole32  1000d6a0     ole32:ole32.dll
 0001:0000c6b4       __IMPORT_DESCRIPTOR_RPCRT4 1000d6b4     rpcrt4:RPCRT4.dll
 0001:0000c6c8       __NULL_IMPORT_DESCRIPTOR   1000d6c8     kernel32:KERNEL32.dll
 0002:00000000       ?OptName@@3UOptionsName@@A 1000f000     FARCmds.obj
 0002:000000b0       ??_R0?AVbad_alloc@std@@@8  1000f0b0     LIBCMT:new.obj
 0002:000000cc       ??_R0?AVexception@std@@@8  1000f0cc     LIBCMT:new.obj
 0002:00000260       ??_R0?AVtype_info@@@8      1000f260     LIBCMT:typinfo.obj
 0002:00000278       ___initialmbcinfo          1000f278     LIBCMT:mbctype.obj
 0002:00000498       __mbctype                  1000f498     LIBCMT:mbctype.obj
 0002:000005a0       __mbcasemap                1000f5a0     LIBCMT:mbctype.obj
 0002:000006a0       ___ptmbcinfo               1000f6a0     LIBCMT:mbctype.obj
 0002:00000798       ___globallocalestatus      1000f798     LIBCMT:glstatus.obj
 0002:0000079c       ___clocalestr              1000f79c     LIBCMT:nlsdata2.obj
 0002:000007a0       ___lc_time_c               1000f7a0     LIBCMT:nlsdata2.obj
 0002:00000908       ___initiallocinfo          1000f908     LIBCMT:nlsdata2.obj
 0002:000009e0       ___ptlocinfo               1000f9e0     LIBCMT:nlsdata2.obj
 0002:000009e4       ___flsindex                1000f9e4     LIBCMT:tidtable.obj
 0002:000009e8       ___getvalueindex           1000f9e8     LIBCMT:tidtable.obj
 0002:000009f8       ___badioinfo               1000f9f8     LIBCMT:ioinit.obj
 0002:00000b60       __cfltcvt_tab              1000fb60     LIBCMT:cmiscdat.obj
 0002:00000b90       ___security_cookie         1000fb90     LIBCMT:gs_cookie.obj
 0002:00000b94       ___security_cookie_complement 1000fb94     LIBCMT:gs_cookie.obj
 0002:00000ba0       ___lconv_static_decimal    1000fba0     LIBCMT:lconv.obj
 0002:00000ba4       ___lconv_static_W_decimal  1000fba4     LIBCMT:lconv.obj
 0002:00000ba8       ___lconv_c                 1000fba8     LIBCMT:lconv.obj
 0002:00000bf8       ___lconv                   1000fbf8     LIBCMT:lconv.obj
 0002:00000bfc       __pctype                   1000fbfc     LIBCMT:ctype.obj
 0002:00000c00       __pwctype                  1000fc00     LIBCMT:ctype.obj
 0002:00000c04       ___mb_cur_max              1000fc04     LIBCMT:nlsdata1.obj
 0002:00000c08       ___decimal_point           1000fc08     LIBCMT:nlsdata1.obj
 0002:00000c0c       ___decimal_point_length    1000fc0c     LIBCMT:nlsdata1.obj
 0002:00000c10       ___abort_behavior          1000fc10     LIBCMT:abort.obj
 0002:00000c20       __NLG_Destination          1000fc20     LIBCMT:exsup.obj
 0002:00000c40       ?Info@@3UPluginStartupInfo@@A 1000fc40     FARCmds.obj
 0002:00000cc8       ?FSF@@3UFarStandardFunctions@@A 1000fcc8     FARCmds.obj
 0002:00000d88       ?Opt@@3UOptions@@A         1000fd88     FARCmds.obj
 0002:0000220c       __aenvptr                  1001120c     LIBCMT:dllcrt0.obj
 0002:00002210       __wenvptr                  10011210     LIBCMT:dllcrt0.obj
 0002:00002214       ___error_mode              10011214     LIBCMT:dllcrt0.obj
 0002:00002218       ___app_type                10011218     LIBCMT:dllcrt0.obj
 0002:0000221c       __crtheap                  1001121c     LIBCMT:heapinit.obj
 0002:00002220       __umaskval                 10011220     LIBCMT:crt0dat.obj
 0002:00002224       ___argc                    10011224     LIBCMT:crt0dat.obj
 0002:00002228       ___argv                    10011228     LIBCMT:crt0dat.obj
 0002:0000222c       ___wargv                   1001122c     LIBCMT:crt0dat.obj
 0002:00002230       __environ                  10011230     LIBCMT:crt0dat.obj
 0002:00002234       ___initenv                 10011234     LIBCMT:crt0dat.obj
 0002:00002238       __wenviron                 10011238     LIBCMT:crt0dat.obj
 0002:0000223c       ___winitenv                1001123c     LIBCMT:crt0dat.obj
 0002:00002240       __pgmptr                   10011240     LIBCMT:crt0dat.obj
 0002:00002244       __wpgmptr                  10011244     LIBCMT:crt0dat.obj
 0002:00002248       __exitflag                 10011248     LIBCMT:crt0dat.obj
 0002:0000224c       __C_Termination_Done       1001124c     LIBCMT:crt0dat.obj
 0002:00002250       __C_Exit_Done              10011250     LIBCMT:crt0dat.obj
 0002:00002880       ?_pnhHeap@@3P6AHI@ZA       10011880     LIBCMT:handler.obj
 0002:00002884       __newmode                  10011884     LIBCMT:_newmode.obj
 0002:0000288c       ___mbulinfo                1001188c     LIBCMT:mbctype.obj
 0002:00002898       ___mbcodepage              10011898     LIBCMT:mbctype.obj
 0002:0000289c       ___ismbcodepage            1001189c     LIBCMT:mbctype.obj
 0002:000028a0       ___mblcid                  100118a0     LIBCMT:mbctype.obj
 0002:000028a4       _gpFlsAlloc                100118a4     LIBCMT:tidtable.obj
 0002:000028a8       _gpFlsGetValue             100118a8     LIBCMT:tidtable.obj
 0002:000028ac       _gpFlsSetValue             100118ac     LIBCMT:tidtable.obj
 0002:000028b0       _gpFlsFree                 100118b0     LIBCMT:tidtable.obj
 0002:000028b4       ___pInvalidArgHandler      100118b4     LIBCMT:invarg.obj
 0002:000028b8       ___locale_changed          100118b8     LIBCMT:setlocal.obj
 0002:000028bc       __maxwait                  100118bc     LIBCMT:crtheap.obj
 0002:00002b18       ?__pInconsistency@@3P6AXXZA 10011b18     LIBCMT:hooks.obj
 0002:00002b34       ___pPurecall               10011b34     LIBCMT:inithelp.obj
 0002:00002b54       ___lconv_static_null       10011b54     LIBCMT:lconv.obj
 0002:00002b58       ___lconv_static_W_null     10011b58     LIBCMT:lconv.obj
 0002:00002e98       ?pArgList@UnDecorator@@0PAVReplicator@@A 10011e98     LIBCMT:undname.obj
 0002:00002e9c       ?pZNameList@UnDecorator@@0PAVReplicator@@A 10011e9c     LIBCMT:undname.obj
 0002:00002ea0       ?pTemplateArgList@UnDecorator@@0PAVReplicator@@A 10011ea0     LIBCMT:undname.obj
 0002:00002ea4       ?gName@UnDecorator@@0PBDB  10011ea4     LIBCMT:undname.obj
 0002:00002ea8       ?name@UnDecorator@@0PBDB   10011ea8     LIBCMT:undname.obj
 0002:00002eac       ?outputString@UnDecorator@@0PADA 10011eac     LIBCMT:undname.obj
 0002:00002eb0       ?maxStringLength@UnDecorator@@0HA 10011eb0     LIBCMT:undname.obj
 0002:00002eb4       ?disableFlags@UnDecorator@@0KA 10011eb4     LIBCMT:undname.obj
 0002:00002eb8       ?m_pGetParameter@UnDecorator@@0P6APADJ@ZA 10011eb8     LIBCMT:undname.obj
 0002:00002ebc       ?fExplicitTemplateParams@UnDecorator@@0_NA 10011ebc     LIBCMT:undname.obj
 0002:00002ebd       ?fGetTemplateArgumentList@UnDecorator@@0_NA 10011ebd     LIBCMT:undname.obj
 0002:00002ec0       __debugger_hook_dummy      10011ec0     <common>
 0002:00002ec4       __pDestructExceptionObject 10011ec4     <common>
 0002:00002ec8       __nhandle                  10011ec8     <common>
 0002:00002ee0       ___pioinfo                 10011ee0     <common>
 0002:00002fe0       ___env_initialized         10011fe0     <common>
 0002:00002fe4       ___onexitend               10011fe4     <common>
 0002:00002fe8       ___onexitbegin             10011fe8     <common>
 0002:00002fec       ___mbctype_initialized     10011fec     <common>
 0002:00002ff0       __FPinit                   10011ff0     <common>
 0002:00002ff4       ___dyn_tls_init_callback   10011ff4     <common>
 0002:00002ff8       ___sse2_available          10011ff8     <common>
 0002:00002ffc       __acmdln                   10011ffc     <common>

 entry point at        0001:00008097

 Static symbols

 0001:00004480       ?GetAlias@@YAPA_WPB_W0@Z   10005480 f   Mix.obj
 0001:00004da0       ?getCurrDir@@YAPA_W_N@Z    10005da0 f   OpenCmd.obj
 0001:00004e00       ?closeHandle@@YAXAAPAX@Z   10005e00 f   OpenCmd.obj
 0001:00004e20       ?killTemp@@YAXPA_W@Z       10005e20 f   OpenCmd.obj
 0001:00004e50       ?createFile@@YAPAXPA_WH@Z  10005e50 f   OpenCmd.obj
 0001:00004ee0       ?createFileStream@@YAXPB_WPAXPAUTShowOutputStreamData@@1@Z 10005ee0 f   OpenCmd.obj
 0001:00004fa0       ?validForView@@YA_NPB_W_N1@Z 10005fa0 f   OpenCmd.obj
 0001:00005190       ?showPartOfOutput@@YAKPAUTShowOutputStreamData@@_N@Z 10006190 f   OpenCmd.obj
 0001:000053e0       ?MakeTempNames@@YA_NPAPA_W0@Z 100063e0 f   OpenCmd.obj
 0001:00005560       ?loadFile@@YAPA_WPB_WKHAAIAA_N@Z 10006560 f   OpenCmd.obj
 0001:00005710       ?GetStreamAndMode@@YAXAAPA_WAAH1@Z 10006710 f   OpenCmd.obj
 0001:000057c0       ?__getContent@@YAPA_WHPA_W@Z 100067c0 f   OpenCmd.obj
 0001:000061a0       ?GetEditParam@@YAPA_WPA_WAAH1AA_N@Z 100071a0 f   OpenCmd.obj
 0001:00006290       ?MakeExecuteString@@YAPB_WPB_W@Z 10007290 f   OpenCmd.obj
 0001:00007fa1       ___DllMainCRTStartup       10008fa1 f   LIBCMT:dllcrt0.obj
 0001:00008397       _doexit                    10009397 f   LIBCMT:crt0dat.obj
 0001:000088a4       __onexit_nolock            100098a4 f   LIBCMT:onexit.obj
 0001:00008ae4       ?CPtoLCID@@YAHH@Z          10009ae4 f   LIBCMT:mbctype.obj
 0001:00008b13       ?setSBCS@@YAXPAUthreadmbcinfostruct@@@Z 10009b13 f   LIBCMT:mbctype.obj
 0001:00008b77       ?setSBUpLow@@YAXPAUthreadmbcinfostruct@@@Z 10009b77 f   LIBCMT:mbctype.obj
 0001:00008dab       ?getSystemCP@@YAHH@Z       10009dab f   LIBCMT:mbctype.obj
 0001:0000a146       _parse_cmdline             1000b146 f   LIBCMT:stdargv.obj
 0001:0000aa8f       _siglookup                 1000ba8f f   LIBCMT:winsig.obj
 0001:0000b3cb       ?__crtLCMapStringA_stat@@YAHPAUlocaleinfo_struct@@KKPBDHPADHHH@Z 1000c3cb f   LIBCMT:a_map.obj
 0001:0000b5f8       ?__crtGetStringTypeA_stat@@YAHPAUlocaleinfo_struct@@KPBDHPAGHHH@Z 1000c5f8 f   LIBCMT:a_str.obj
 0001:0000be12       ?x_ismbbtype_l@@YAHPAUlocaleinfo_struct@@IHH@Z 1000ce12 f   LIBCMT:ismbbyte.obj
 0001:0000bf10       __unwind_handler4          1000cf10 f   LIBCMT:exsup4.obj
 0001:0000c170       __unwind_handler           1000d170 f   LIBCMT:exsup.obj
 0001:0000c429       ??__Fnomem@?5???2@YAPAXI@Z@YAXXZ 1000d429 f   LIBCMT:new.obj
